 net

 Timestamp is 68fa8ffc (Thu Oct 23 20:28:44 2025)

 Preferred load address is 10000000

 Start         Length     Name                   Class
 0001:00000000 0000c942H .text$mn                CODE
 0002:00000000 00000208H .idata$5                DATA
 0002:00000208 00000008H .00cfg                  DATA
 0002:00000210 00000004H .CRT$XCA                DATA
 0002:00000214 00000004H .CRT$XCZ                DATA
 0002:00000218 00000004H .CRT$XIA                DATA
 0002:0000021c 00000004H .CRT$XIZ                DATA
 0002:00000220 00000004H .CRT$XPA                DATA
 0002:00000224 00000004H .CRT$XPZ                DATA
 0002:00000228 00000004H .CRT$XTA                DATA
 0002:0000022c 00000004H .CRT$XTZ                DATA
 0002:00000230 00000000H .gfids$y                DATA
 0002:00000230 00001f90H .rdata                  DATA
 0002:000021c0 00000000H .rdata$CastGuardVftablesA DATA
 0002:000021c0 00000000H .rdata$CastGuardVftablesC DATA
 0002:000021c0 00000004H .rdata$sxdata           DATA
 0002:000021c4 00000078H .rdata$voltmd           DATA
 0002:0000223c 0000035cH .rdata$zzzdbg           DATA
 0002:00002598 00000004H .rtc$IAA                DATA
 0002:0000259c 00000004H .rtc$IZZ                DATA
 0002:000025a0 00000004H .rtc$TAA                DATA
 0002:000025a4 00000004H .rtc$TZZ                DATA
 0002:000025a8 00000084H .xdata$x                DATA
 0002:0000262c 00000040H .didat$2                DATA
 0002:0000266c 00000020H .didat$3                DATA
 0002:0000268c 0000004cH .didat$4                DATA
 0002:000026d8 0000015cH .didat$6                DATA
 0002:00002834 0000004cH .didat$7                DATA
 0002:00002880 000021e0H .edata                  DATA
 0002:00004a60 000000c8H .idata$2                DATA
 0002:00004b28 00000014H .idata$3                DATA
 0002:00004b3c 00000208H .idata$4                DATA
 0002:00004d44 000007c6H .idata$6                DATA
 0003:00000000 000000a8H .data                   DATA
 0003:000000a8 00000050H .didat$5                DATA
 0003:000000f8 0000056cH .bss                    DATA
 0004:00000000 00000060H .rsrc$01                DATA
 0004:00000060 00000328H .rsrc$02                DATA

  Address         Publics by Value              Rva+Base       Lib:Object

 0000:00000000       ___AbsoluteZero            00000000     <absolute>
 0000:00000000       ___arm64x_extra_rfe_table  00000000     <absolute>
 0000:00000000       ___arm64x_extra_rfe_table_size 00000000     <absolute>
 0000:00000000       ___arm64x_native_entrypoint 00000000     <absolute>
 0000:00000000       ___arm64x_redirection_metadata 00000000     <absolute>
 0000:00000000       ___arm64x_redirection_metadata_count 00000000     <absolute>
 0000:00000000       ___dynamic_value_reloc_table 00000000     <absolute>
 0000:00000000       ___enclave_config          00000000     <absolute>
 0000:00000000       ___guard_check_icall_a64n_fptr 00000000     <absolute>
 0000:00000000       ___guard_eh_cont_count     00000000     <absolute>
 0000:00000000       ___guard_eh_cont_table     00000000     <absolute>
 0000:00000000       ___guard_fids_count        00000000     <absolute>
 0000:00000000       ___guard_fids_table        00000000     <absolute>
 0000:00000000       ___guard_iat_count         00000000     <absolute>
 0000:00000000       ___guard_iat_table         00000000     <absolute>
 0000:00000000       ___guard_longjmp_count     00000000     <absolute>
 0000:00000000       ___guard_longjmp_table     00000000     <absolute>
 0000:00000000       ___hybrid_auxiliary_delayload_iat 00000000     <absolute>
 0000:00000000       ___hybrid_auxiliary_delayload_iat_copy 00000000     <absolute>
 0000:00000000       ___hybrid_auxiliary_iat    00000000     <absolute>
 0000:00000000       ___hybrid_auxiliary_iat_copy 00000000     <absolute>
 0000:00000000       ___hybrid_code_map         00000000     <absolute>
 0000:00000000       ___hybrid_code_map_count   00000000     <absolute>
 0000:00000000       ___hybrid_image_info_bitfield 00000000     <absolute>
 0000:00000000       ___x64_code_ranges_to_entry_points 00000000     <absolute>
 0000:00000000       ___x64_code_ranges_to_entry_points_count 00000000     <absolute>
 0000:00000001       ___safe_se_handler_count   00000001     <absolute>
 0000:00000100       ___guard_flags             00000100     <absolute>
 0000:00000000       ___ImageBase               10000000     <linker-defined>
 0001:00000000       _Java_java_net_DatagramPacket_init@8 10001000 f   DatagramPacket.obj
 0001:000000b4       _Java_sun_net_spi_DefaultProxySelector_getSystemProxy@16 100010b4 f   DefaultProxySelector.obj
 0001:0000045d       _Java_sun_net_spi_DefaultProxySelector_init@8 1000145d f   DefaultProxySelector.obj
 0001:000005c4       ___local_stdio_printf_options 100015c4 f i DefaultProxySelector.obj
 0001:000005ca       ___local_stdio_scanf_options 100015ca f i DefaultProxySelector.obj
 0001:000005d0       __vfprintf_l               100015d0 f i DefaultProxySelector.obj
 0001:000005f4       __vsnprintf_l              100015f4 f i DefaultProxySelector.obj
 0001:00000627       __vsscanf_l                10001627 f i DefaultProxySelector.obj
 0001:0000064d       _fprintf                   1000164d f i DefaultProxySelector.obj
 0001:00000665       _sprintf                   10001665 f i DefaultProxySelector.obj
 0001:0000067f       _sscanf                    1000167f f i DefaultProxySelector.obj
 0001:00000697       _Java_java_net_DualStackPlainDatagramSocketImpl_dataAvailable@8 10001697 f   DualStackPlainDatagramSocketImpl.obj
 0001:00000701       _Java_java_net_DualStackPlainDatagramSocketImpl_initIDs@8 10001701 f   DualStackPlainDatagramSocketImpl.obj
 0001:0000074d       _Java_java_net_DualStackPlainDatagramSocketImpl_socketBind@24 1000174d f   DualStackPlainDatagramSocketImpl.obj
 0001:000007d3       _Java_java_net_DualStackPlainDatagramSocketImpl_socketClose@12 100017d3 f   DualStackPlainDatagramSocketImpl.obj
 0001:000007d3       _Java_java_net_DualStackPlainSocketImpl_close0@12 100017d3 f   DualStackPlainSocketImpl.obj
 0001:000007df       _Java_java_net_DualStackPlainDatagramSocketImpl_socketConnect@20 100017df f   DualStackPlainDatagramSocketImpl.obj
 0001:00000874       _Java_java_net_DualStackPlainDatagramSocketImpl_socketCreate@12 10001874 f   DualStackPlainDatagramSocketImpl.obj
 0001:0000092c       _Java_java_net_DualStackPlainDatagramSocketImpl_socketDisconnect@12 1000192c f   DualStackPlainDatagramSocketImpl.obj
 0001:0000098f       _Java_java_net_DualStackPlainDatagramSocketImpl_socketGetIntOption@16 1000198f f   DualStackPlainDatagramSocketImpl.obj
 0001:00000a09       _Java_java_net_DualStackPlainDatagramSocketImpl_socketLocalAddress@12 10001a09 f   DualStackPlainDatagramSocketImpl.obj
 0001:00000a6d       _Java_java_net_DualStackPlainDatagramSocketImpl_socketLocalPort@12 10001a6d f   DualStackPlainDatagramSocketImpl.obj
 0001:00000ad0       _Java_java_net_DualStackPlainDatagramSocketImpl_socketReceiveOrPeekData@28 10001ad0 f   DualStackPlainDatagramSocketImpl.obj
 0001:00000e21       _Java_java_net_DualStackPlainDatagramSocketImpl_socketSend@36 10001e21 f   DualStackPlainDatagramSocketImpl.obj
 0001:00000f3a       _Java_java_net_DualStackPlainDatagramSocketImpl_socketSetIntOption@20 10001f3a f   DualStackPlainDatagramSocketImpl.obj
 0001:00001065       _Java_java_net_DualStackPlainSocketImpl_accept0@16 10002065 f   DualStackPlainSocketImpl.obj
 0001:0000113c       _Java_java_net_DualStackPlainSocketImpl_available0@12 1000213c f   DualStackPlainSocketImpl.obj
 0001:00001176       _Java_java_net_DualStackPlainSocketImpl_bind0@24 10002176 f   DualStackPlainSocketImpl.obj
 0001:000011e4       _Java_java_net_DualStackPlainSocketImpl_configureBlocking@16 100021e4 f   DualStackPlainSocketImpl.obj
 0001:00001222       _Java_java_net_DualStackPlainSocketImpl_connect0@20 10002222 f   DualStackPlainSocketImpl.obj
 0001:000012b6       _Java_java_net_DualStackPlainSocketImpl_getIntOption@16 100022b6 f   DualStackPlainSocketImpl.obj
 0001:0000135c       _Java_java_net_DualStackPlainSocketImpl_initIDs@8 1000235c f   DualStackPlainSocketImpl.obj
 0001:000013ae       _Java_java_net_DualStackPlainSocketImpl_listen0@16 100023ae f   DualStackPlainSocketImpl.obj
 0001:000013d9       _Java_java_net_DualStackPlainSocketImpl_localAddress@16 100023d9 f   DualStackPlainSocketImpl.obj
 0001:00001473       _Java_java_net_DualStackPlainSocketImpl_localPort0@12 10002473 f   DualStackPlainSocketImpl.obj
 0001:000014f5       _Java_java_net_DualStackPlainSocketImpl_sendOOB@16 100024f5 f   DualStackPlainSocketImpl.obj
 0001:0000153c       _Java_java_net_DualStackPlainSocketImpl_setIntOption@20 1000253c f   DualStackPlainSocketImpl.obj
 0001:000015c7       _Java_java_net_DualStackPlainSocketImpl_shutdown0@16 100025c7 f   DualStackPlainSocketImpl.obj
 0001:000015d8       _Java_java_net_DualStackPlainSocketImpl_socket0@16 100025d8 f   DualStackPlainSocketImpl.obj
 0001:00001652       _Java_java_net_DualStackPlainSocketImpl_waitForConnect@16 10002652 f   DualStackPlainSocketImpl.obj
 0001:0000176d       _Java_java_net_DualStackPlainSocketImpl_waitForNewConnection@16 1000276d f   DualStackPlainSocketImpl.obj
 0001:000017b7       _Java_sun_net_ExtendedOptionsImpl_flowSupported@8 100027b7 f   ExtendedOptionsImpl.obj
 0001:000017b7       _Java_sun_net_ExtendedOptionsImpl_keepAliveOptionsSupported@8 100027b7 f   ExtendedOptionsImpl.obj
 0001:000017bc       _Java_sun_net_ExtendedOptionsImpl_getFlowOption@16 100027bc f   ExtendedOptionsImpl.obj
 0001:000017bc       _Java_sun_net_ExtendedOptionsImpl_setFlowOption@16 100027bc f   ExtendedOptionsImpl.obj
 0001:000017bc       _Java_sun_net_ExtendedOptionsImpl_setTcpKeepAliveIntvl@16 100027bc f   ExtendedOptionsImpl.obj
 0001:000017bc       _Java_sun_net_ExtendedOptionsImpl_setTcpKeepAliveProbes@16 100027bc f   ExtendedOptionsImpl.obj
 0001:000017bc       _Java_sun_net_ExtendedOptionsImpl_setTcpKeepAliveTime@16 100027bc f   ExtendedOptionsImpl.obj
 0001:000017d2       _Java_sun_net_ExtendedOptionsImpl_getTcpKeepAliveIntvl@12 100027d2 f   ExtendedOptionsImpl.obj
 0001:000017d2       _Java_sun_net_ExtendedOptionsImpl_getTcpKeepAliveProbes@12 100027d2 f   ExtendedOptionsImpl.obj
 0001:000017d2       _Java_sun_net_ExtendedOptionsImpl_getTcpKeepAliveTime@12 100027d2 f   ExtendedOptionsImpl.obj
 0001:000017e8       _Java_sun_net_ExtendedOptionsImpl_init@8 100027e8 f   ExtendedOptionsImpl.obj
 0001:000017eb       _Java_java_net_Inet4Address_init@8 100027eb f   Inet4Address.obj
 0001:00001843       _Java_java_net_Inet4AddressImpl_getHostByAddr@12 10002843 f   Inet4AddressImpl.obj
 0001:000018c0       _Java_java_net_Inet4AddressImpl_getLocalHostName@8 100028c0 f   Inet4AddressImpl.obj
 0001:000018c0       _Java_java_net_Inet6AddressImpl_getLocalHostName@8 100028c0 f   Inet6AddressImpl.obj
 0001:0000191d       _Java_java_net_Inet4AddressImpl_isReachable0@24 1000291d f   Inet4AddressImpl.obj
 0001:00001a6c       _Java_java_net_Inet4AddressImpl_lookupAllHostAddr@12 10002a6c f   Inet4AddressImpl.obj
 0001:00001d85       _isDottedIPAddress         10002d85 f   Inet4AddressImpl.obj
 0001:0000222c       _Java_java_net_Inet6Address_init@8 1000322c f   Inet6Address.obj
 0001:0000236f       _Java_java_net_Inet6AddressImpl_getHostByAddr@12 1000336f f   Inet6AddressImpl.obj
 0001:0000249b       _Java_java_net_Inet6AddressImpl_isReachable0@32 1000349b f   Inet6AddressImpl.obj
 0001:00002635       _Java_java_net_Inet6AddressImpl_lookupAllHostAddr@12 10003635 f   Inet6AddressImpl.obj
 0001:00002c56       _Java_java_net_InetAddress_init@8 10003c56 f   InetAddress.obj
 0001:00002d94       _Java_java_net_InetAddressImplFactory_isIPv6Supported@8 10003d94 f   InetAddressImplFactory.obj
 0001:00002da1       _Java_sun_net_www_protocol_http_ntlm_NTLMAuthSequence_getCredentialsHandle@20 10003da1 f   NTLMAuthSequence.obj
 0001:00002f3c       _Java_sun_net_www_protocol_http_ntlm_NTLMAuthSequence_getNextToken@24 10003f3c f   NTLMAuthSequence.obj
 0001:00003176       _Java_sun_net_www_protocol_http_ntlm_NTLMAuthSequence_initFirst@12 10004176 f   NTLMAuthSequence.obj
 0001:00003224       _Java_sun_net_www_protocol_http_ntlm_NTLMAuthentication_isTrustedSite0@12 10004224 f   NTLMAuthentication.obj
 0001:000032f7       _Java_sun_net_www_protocol_http_ntlm_NTLMAuthentication_isTrustedSiteAvailable@8 100042f7 f   NTLMAuthentication.obj
 0001:00003323       _Java_java_net_NetworkInterface_getAll@8 10004323 f   NetworkInterface.obj
 0001:000033d2       _Java_java_net_NetworkInterface_getByIndex0@12 100043d2 f   NetworkInterface.obj
 0001:00003439       _Java_java_net_NetworkInterface_getByInetAddress0@12 10004439 f   NetworkInterface.obj
 0001:0000350a       _Java_java_net_NetworkInterface_getByName0@12 1000450a f   NetworkInterface.obj
 0001:000035c9       _Java_java_net_NetworkInterface_getMTU0@16 100045c9 f   NetworkInterface.obj
 0001:00003602       _Java_java_net_NetworkInterface_getMacAddr0@20 10004602 f   NetworkInterface.obj
 0001:00003697       _Java_java_net_NetworkInterface_init@8 10004697 f   NetworkInterface.obj
 0001:0000386c       _Java_java_net_NetworkInterface_isLoopback0@16 1000486c f   NetworkInterface.obj
 0001:000038ac       _Java_java_net_NetworkInterface_isP2P0@16 100048ac f   NetworkInterface.obj
 0001:000038f0       _Java_java_net_NetworkInterface_isUp0@16 100048f0 f   NetworkInterface.obj
 0001:0000393d       _Java_java_net_NetworkInterface_supportsMulticast0@16 1000493d f   NetworkInterface.obj
 0001:00003942       __snprintf_s               10004942 f i NetworkInterface.obj
 0001:00003961       __vsnprintf_s_l            10004961 f i NetworkInterface.obj
 0001:00003993       _createNetworkInterface    10004993 f   NetworkInterface.obj
 0001:00003d85       _enumAddresses_win         10004d85 f   NetworkInterface.obj
 0001:00003f79       _enumInterfaces            10004f79 f   NetworkInterface.obj
 0001:00004452       _free_netaddr              10005452 f   NetworkInterface.obj
 0001:0000446c       _free_netif                1000546c f   NetworkInterface.obj
 0001:000044b5       _getIF                     100054b5 f   NetworkInterface.obj
 0001:0000457f       _Java_java_net_NetworkInterface_getAll_XP@8 1000557f f   NetworkInterface_winXP.obj
 0001:0000460b       _Java_java_net_NetworkInterface_getByIndex0_XP@12 1000560b f   NetworkInterface_winXP.obj
 0001:00004662       _Java_java_net_NetworkInterface_getByInetAddress0_XP@12 10005662 f   NetworkInterface_winXP.obj
 0001:000046cc       _Java_java_net_NetworkInterface_getByName0_XP@12 100056cc f   NetworkInterface_winXP.obj
 0001:0000474e       _Java_java_net_NetworkInterface_getMTU0_XP@16 1000574e f   NetworkInterface_winXP.obj
 0001:00004776       _Java_java_net_NetworkInterface_getMacAddr0_XP@16 10005776 f   NetworkInterface_winXP.obj
 0001:000047cb       _Java_java_net_NetworkInterface_isLoopback0_XP@16 100057cb f   NetworkInterface_winXP.obj
 0001:000047f6       _Java_java_net_NetworkInterface_isP2P0_XP@16 100057f6 f   NetworkInterface_winXP.obj
 0001:00004831       _Java_java_net_NetworkInterface_isUp0_XP@16 10005831 f   NetworkInterface_winXP.obj
 0001:0000485c       _Java_java_net_NetworkInterface_supportsMulticast0_XP@16 1000585c f   NetworkInterface_winXP.obj
 0001:00004c04       _getAdapter                10005c04 f   NetworkInterface_winXP.obj
 0001:00004f50       _getAllInterfacesAndAddresses 10005f50 f   NetworkInterface_winXP.obj
 0001:000051e8       _Java_sun_net_dns_ResolverConfigurationImpl_init0@8 100061e8 f   ResolverConfigurationImpl.obj
 0001:0000522c       _Java_sun_net_dns_ResolverConfigurationImpl_loadDNSconfig0@8 1000622c f   ResolverConfigurationImpl.obj
 0001:000052d6       _Java_sun_net_dns_ResolverConfigurationImpl_notifyAddrChange0@8 100062d6 f   ResolverConfigurationImpl.obj
 0001:000056c0       _Java_java_net_SocketInputStream_init@8 100066c0 f   SocketInputStream.obj
 0001:000056d2       _Java_java_net_SocketInputStream_socketRead0@28 100066d2 f   SocketInputStream.obj
 0001:000058f4       _Java_java_net_SocketOutputStream_init@8 100068f4 f   SocketOutputStream.obj
 0001:00005906       _Java_java_net_SocketOutputStream_socketWrite0@24 10006906 f   SocketOutputStream.obj
 0001:00005af9       _Java_java_net_TwoStacksPlainDatagramSocketImpl_bind0@20 10006af9 f   TwoStacksPlainDatagramSocketImpl.obj
 0001:00005daf       _Java_java_net_TwoStacksPlainDatagramSocketImpl_connect0@16 10006daf f   TwoStacksPlainDatagramSocketImpl.obj
 0001:00005f37       _Java_java_net_TwoStacksPlainDatagramSocketImpl_dataAvailable@8 10006f37 f   TwoStacksPlainDatagramSocketImpl.obj
 0001:00005ff6       _Java_java_net_TwoStacksPlainDatagramSocketImpl_datagramSocketClose@8 10006ff6 f   TwoStacksPlainDatagramSocketImpl.obj
 0001:000060a7       _Java_java_net_TwoStacksPlainDatagramSocketImpl_datagramSocketCreate@8 100070a7 f   TwoStacksPlainDatagramSocketImpl.obj
 0001:0000622e       _Java_java_net_TwoStacksPlainDatagramSocketImpl_disconnect0@12 1000722e f   TwoStacksPlainDatagramSocketImpl.obj
 0001:000062e6       _Java_java_net_TwoStacksPlainDatagramSocketImpl_getTTL@8 100072e6 f   TwoStacksPlainDatagramSocketImpl.obj
 0001:000062eb       _Java_java_net_TwoStacksPlainDatagramSocketImpl_getTimeToLive@8 100072eb f   TwoStacksPlainDatagramSocketImpl.obj
 0001:000063c9       _Java_java_net_TwoStacksPlainDatagramSocketImpl_init@8 100073c9 f   TwoStacksPlainDatagramSocketImpl.obj
 0001:0000659d       _Java_java_net_TwoStacksPlainDatagramSocketImpl_join@16 1000759d f   TwoStacksPlainDatagramSocketImpl.obj
 0001:000065ba       _Java_java_net_TwoStacksPlainDatagramSocketImpl_leave@16 100075ba f   TwoStacksPlainDatagramSocketImpl.obj
 0001:000065d7       _Java_java_net_TwoStacksPlainDatagramSocketImpl_peek@12 100075d7 f   TwoStacksPlainDatagramSocketImpl.obj
 0001:00006822       _Java_java_net_TwoStacksPlainDatagramSocketImpl_peekData@12 10007822 f   TwoStacksPlainDatagramSocketImpl.obj
 0001:00006cab       _Java_java_net_TwoStacksPlainDatagramSocketImpl_receive0@12 10007cab f   TwoStacksPlainDatagramSocketImpl.obj
 0001:0000712a       _Java_java_net_TwoStacksPlainDatagramSocketImpl_send@12 1000812a f   TwoStacksPlainDatagramSocketImpl.obj
 0001:000073ec       _Java_java_net_TwoStacksPlainDatagramSocketImpl_setTTL@12 100083ec f   TwoStacksPlainDatagramSocketImpl.obj
 0001:00007402       _Java_java_net_TwoStacksPlainDatagramSocketImpl_setTimeToLive@12 10008402 f   TwoStacksPlainDatagramSocketImpl.obj
 0001:000074d8       _Java_java_net_TwoStacksPlainDatagramSocketImpl_socketGetOption@12 100084d8 f   TwoStacksPlainDatagramSocketImpl.obj
 0001:0000768c       _Java_java_net_TwoStacksPlainDatagramSocketImpl_socketLocalAddress@12 1000868c f   TwoStacksPlainDatagramSocketImpl.obj
 0001:00007767       _Java_java_net_TwoStacksPlainDatagramSocketImpl_socketNativeSetOption@16 10008767 f   TwoStacksPlainDatagramSocketImpl.obj
 0001:000079ab       _createBoolean             100089ab f   TwoStacksPlainDatagramSocketImpl.obj
 0001:00007a1d       _createInteger             10008a1d f   TwoStacksPlainDatagramSocketImpl.obj
 0001:00007a89       _exceedSizeLimit           10008a89 f   TwoStacksPlainDatagramSocketImpl.obj
 0001:0000805c       _getMulticastInterface     1000905c f   TwoStacksPlainDatagramSocketImpl.obj
 0001:00008930       _IN6_IS_ADDR_UNSPECIFIED   10009930 f i TwoStacksPlainSocketImpl.obj
 0001:00008968       _Java_java_net_TwoStacksPlainSocketImpl_initProto@8 10009968 f   TwoStacksPlainSocketImpl.obj
 0001:00008aa5       _Java_java_net_TwoStacksPlainSocketImpl_socketAccept@12 10009aa5 f   TwoStacksPlainSocketImpl.obj
 0001:00008f17       _Java_java_net_TwoStacksPlainSocketImpl_socketAvailable@8 10009f17 f   TwoStacksPlainSocketImpl.obj
 0001:00008f88       _Java_java_net_TwoStacksPlainSocketImpl_socketBind@20 10009f88 f   TwoStacksPlainSocketImpl.obj
 0001:0000923b       _Java_java_net_TwoStacksPlainSocketImpl_socketClose0@12 1000a23b f   TwoStacksPlainSocketImpl.obj
 0001:000092fe       _Java_java_net_TwoStacksPlainSocketImpl_socketConnect@20 1000a2fe f   TwoStacksPlainSocketImpl.obj
 0001:00009778       _Java_java_net_TwoStacksPlainSocketImpl_socketCreate@12 1000a778 f   TwoStacksPlainSocketImpl.obj
 0001:000098af       _Java_java_net_TwoStacksPlainSocketImpl_socketGetOption@16 1000a8af f   TwoStacksPlainSocketImpl.obj
 0001:00009a8b       _Java_java_net_TwoStacksPlainSocketImpl_socketListen@12 1000aa8b f   TwoStacksPlainSocketImpl.obj
 0001:00009c05       _Java_java_net_TwoStacksPlainSocketImpl_socketNativeSetOption@20 1000ac05 f   TwoStacksPlainSocketImpl.obj
 0001:00009ead       _Java_java_net_TwoStacksPlainSocketImpl_socketSendUrgentData@12 1000aead f   TwoStacksPlainSocketImpl.obj
 0001:00009f24       _Java_java_net_TwoStacksPlainSocketImpl_socketShutdown@12 1000af24 f   TwoStacksPlainSocketImpl.obj
 0001:00009fdd       _JNI_OnLoad@8              1000afdd f   net_util.obj
 0001:0000a0a3       _NET_SockaddrEqualsInetAddress@12 1000b0a3 f   net_util.obj
 0001:0000a1af       _NET_SockaddrToInetAddress@12 1000b1af f   net_util.obj
 0001:0000a2ff       _getInet6Address_ipaddress 1000b2ff f   net_util.obj
 0001:0000a34a       _getInet6Address_scopeid   1000b34a f   net_util.obj
 0001:0000a37f       _getInetAddress_addr       1000b37f f   net_util.obj
 0001:0000a3bf       _getInetAddress_family     1000b3bf f   net_util.obj
 0001:0000a3ff       _initInetAddressIDs@4      1000b3ff f   net_util.obj
 0001:0000a45a       _ipv6_available@0          1000b45a f   net_util.obj
 0001:0000a460       _setInet6Address_ipaddress 1000b460 f   net_util.obj
 0001:0000a4d5       _setInet6Address_scopeid   1000b4d5 f   net_util.obj
 0001:0000a527       _setInet6Address_scopeifname 1000b527 f   net_util.obj
 0001:0000a560       _setInetAddress_addr       1000b560 f   net_util.obj
 0001:0000a5a1       _setInetAddress_family     1000b5a1 f   net_util.obj
 0001:0000a5e2       _setInetAddress_hostName   1000b5e2 f   net_util.obj
 0001:0000a639       _DllMain@12                1000b639 f   net_util_md.obj
 0001:0000a68a       _IN6ADDR_SETANY            1000b68a f i net_util_md.obj
 0001:0000a6b3       _IN6_IS_ADDR_LINKLOCAL     1000b6b3 f i net_util_md.obj
 0001:0000a6cb       _IPv6_supported            1000b6cb f   net_util_md.obj
 0001:0000a6ea       _NET_Bind@12               1000b6ea f   net_util_md.obj
 0001:0000a722       _NET_BindV6@8              1000b722 f   net_util_md.obj
 0001:0000aa7d       _NET_EnableFastTcpLoopback@4 1000ba7d f   net_util_md.obj
 0001:0000aac0       _NET_GetDefaultTOS         1000bac0 f   net_util_md.obj
 0001:0000ab87       _NET_GetFileDescriptorID   1000bb87 f   net_util_md.obj
 0001:0000abb5       _NET_GetPortFromSockaddr@4 1000bbb5 f   net_util_md.obj
 0001:0000abca       _NET_GetSockOpt@20         1000bbca f   net_util_md.obj
 0001:0000ac35       _NET_IPv4MappedToIPv4      1000bc35 f   net_util_md.obj
 0001:0000ac59       _NET_InetAddressToSockaddr@24 1000bc59 f   net_util_md.obj
 0001:0000ae49       _NET_IsEqual               1000be49 f   net_util_md.obj
 0001:0000ae6d       _NET_IsIPv4Mapped          1000be6d f   net_util_md.obj
 0001:0000ae92       _NET_MapSocketOption@12    1000be92 f   net_util_md.obj
 0001:0000aed1       _NET_MapSocketOptionV6@12  1000bed1 f   net_util_md.obj
 0001:0000af19       _NET_SetSockOpt@20         1000bf19 f   net_util_md.obj
 0001:0000afbf       _NET_Socket                1000bfbf f   net_util_md.obj
 0001:0000afe8       _NET_SocketClose@4         1000bfe8 f   net_util_md.obj
 0001:0000b035       _NET_ThrowByNameWithLastError 1000c035 f   net_util_md.obj
 0001:0000b047       _NET_ThrowCurrent          1000c047 f   net_util_md.obj
 0001:0000b05c       _NET_ThrowNew@12           1000c05c f   net_util_md.obj
 0001:0000b13f       _NET_ThrowSocketException  1000c13f f   net_util_md.obj
 0001:0000b181       _NET_Timeout2@16           1000c181 f   net_util_md.obj
 0001:0000b258       _NET_Timeout@8             1000c258 f   net_util_md.obj
 0001:0000b2c8       _NET_Wait                  1000c2c8 f   net_util_md.obj
 0001:0000b422       _NET_WinBind@16            1000c422 f   net_util_md.obj
 0001:0000b446       _cmpScopeID                1000c446 f   net_util_md.obj
 0001:0000b457       _getDefaultIPv6Interface   1000c457 f   net_util_md.obj
 0001:0000b4c5       _getScopeID                1000c4c5 f   net_util_md.obj
 0001:0000b4cd       @_guard_check_icall_nop@4  1000c4cd f   MSVCRT:guard_support.obj
 0001:0000b4cd       _parseExclusiveBindProperty 1000c4cd f   net_util_md.obj
 0001:0000b4cd       _platformInit              1000c4cd f   net_util_md.obj
 0001:0000b4d0       _setExclusiveBind          1000c4d0 f   net_util_md.obj
 0001:0000b51c       _Java_sun_net_PortConfig_getLower0@8 1000c51c f   portconfig.obj
 0001:0000b532       _Java_sun_net_PortConfig_getUpper0@8 1000c532 f   portconfig.obj
 0001:0000b5ff       ___WSAFDIsSet@8            1000c5ff f   ws2_32:WS2_32.dll
 0001:0000b605       _JVM_CurrentTimeMillis@8   1000c605 f   jvm:jvm.dll
 0001:0000b60b       _JVM_InitializeSocketLibrary@0 1000c60b f   jvm:jvm.dll
 0001:0000b611       _jio_snprintf              1000c611 f   jvm:jvm.dll
 0001:0000b617       __imp_load__AcquireCredentialsHandleA@36 1000c617 f   secur32:Secur32.dll
 0001:0000b621       _AcquireCredentialsHandleA@36 1000c621 f   secur32:Secur32.dll
 0001:0000b627       __tailMerge_secur32_dll    1000c627     secur32:Secur32.dll
 0001:0000b638       __imp_load__FreeCredentialsHandle@4 1000c638 f   secur32:Secur32.dll
 0001:0000b642       __imp_load__InitializeSecurityContextA@48 1000c642 f   secur32:Secur32.dll
 0001:0000b64c       _InitializeSecurityContextA@48 1000c64c f   secur32:Secur32.dll
 0001:0000b652       __imp_load__CompleteAuthToken@8 1000c652 f   secur32:Secur32.dll
 0001:0000b65c       _CompleteAuthToken@8       1000c65c f   secur32:Secur32.dll
 0001:0000b662       __imp_load__DeleteSecurityContext@4 1000c662 f   secur32:Secur32.dll
 0001:0000b66c       __imp_load__IcmpCreateFile@0 1000c66c f   iphlpapi:IPHLPAPI.DLL
 0001:0000b676       __tailMerge_iphlpapi_dll   1000c676     iphlpapi:IPHLPAPI.DLL
 0001:0000b687       __imp_load__IcmpCloseHandle@4 1000c687 f   iphlpapi:IPHLPAPI.DLL
 0001:0000b691       __imp_load__IcmpSendEcho@32 1000c691 f   iphlpapi:IPHLPAPI.DLL
 0001:0000b69b       __imp_load__IcmpSendEcho2Ex@48 1000c69b f   iphlpapi:IPHLPAPI.DLL
 0001:0000b6a5       __imp_load__Icmp6CreateFile@0 1000c6a5 f   iphlpapi:IPHLPAPI.DLL
 0001:0000b6af       __imp_load__Icmp6SendEcho2@48 1000c6af f   iphlpapi:IPHLPAPI.DLL
 0001:0000b6b9       __imp_load__GetIfTable@12  1000c6b9 f   iphlpapi:IPHLPAPI.DLL
 0001:0000b6c3       __imp_load__GetIpAddrTable@12 1000c6c3 f   iphlpapi:IPHLPAPI.DLL
 0001:0000b6cd       __imp_load__GetFriendlyIfIndex@4 1000c6cd f   iphlpapi:IPHLPAPI.DLL
 0001:0000b6d7       __imp_load__GetAdaptersAddresses@20 1000c6d7 f   iphlpapi:IPHLPAPI.DLL
 0001:0000b6e1       __imp_load__NotifyAddrChange@8 1000c6e1 f   iphlpapi:IPHLPAPI.DLL
 0001:0000b6eb       __imp_load__GetAdaptersInfo@8 1000c6eb f   iphlpapi:IPHLPAPI.DLL
 0001:0000b6f5       ?DloadAcquireSectionWriteAccess@@YGXXZ 1000c6f5 f i delayimp:delayhlp.obj
 0001:0000b728       ?DloadGetSRWLockFunctionPointers@@YGEXZ 1000c728 f i delayimp:delayhlp.obj
 0001:0000b79e       ?DloadLock@@YGXXZ          1000c79e f i delayimp:delayhlp.obj
 0001:0000b7dd       ?DloadMakePermanentImageCommit@@YGXPAXK@Z 1000c7dd f i delayimp:delayhlp.obj
 0001:0000b84c       ?DloadObtainSection@@YGPAXPAK0@Z 1000c84c f i delayimp:delayhlp.obj
 0001:0000b8c7       ?DloadProtectSection@@YGXKPAK@Z 1000c8c7 f i delayimp:delayhlp.obj
 0001:0000b935       ?DloadReleaseSectionWriteAccess@@YGXXZ 1000c935 f i delayimp:delayhlp.obj
 0001:0000b96b       ?DloadUnlock@@YGXXZ        1000c96b f i delayimp:delayhlp.obj
 0001:0000b997       ___delayLoadHelper2@8      1000c997 f   delayimp:delayhlp.obj
 0001:0000bc06       _JNU_ThrowOutOfMemoryError@8 1000cc06 f   java:java.dll
 0001:0000bc0c       _JNU_ThrowByName@12        1000cc0c f   java:java.dll
 0001:0000bc12       _JNU_ThrowByNameWithLastError@12 1000cc12 f   java:java.dll
 0001:0000bc18       _JNU_ThrowNullPointerException@8 1000cc18 f   java:java.dll
 0001:0000bc1e       _JNU_NewStringPlatform@8   1000cc1e f   java:java.dll
 0001:0000bc24       _JNU_GetStringPlatformChars@12 1000cc24 f   java:java.dll
 0001:0000bc2a       _JNU_ReleaseStringPlatformChars@12 1000cc2a f   java:java.dll
 0001:0000bc30       _JDK_LoadSystemLibrary     1000cc30 f   java:java.dll
 0001:0000bc36       _getErrorString            1000cc36 f   java:java.dll
 0001:0000bc3c       _JNU_ThrowByNameWithMessageAndLastError@12 1000cc3c f   java:java.dll
 0001:0000bc42       @__security_check_cookie@4 1000cc42 f   MSVCRT:secchk.obj
 0001:0000bf90       __DllMainCRTStartup@12     1000cf90 f   MSVCRT:dll_dllmain.obj
 0001:0000bfb3       ___raise_securityfailure   1000cfb3 f   MSVCRT:gs_report.obj
 0001:0000bfdb       ___report_gsfailure        1000cfdb f   MSVCRT:gs_report.obj
 0001:0000c122       ___security_init_cookie    1000d122 f   MSVCRT:gs_support.obj
 0001:0000c16d       ?__scrt_initialize_type_info@@YAXXZ 1000d16d f   MSVCRT:tncleanup.obj
 0001:0000c179       ?__scrt_uninitialize_type_info@@YAXXZ 1000d179 f   MSVCRT:tncleanup.obj
 0001:0000c185       ___scrt_initialize_default_local_stdio_options 1000d185 f   MSVCRT:default_local_stdio_options.obj
 0001:0000c1e6       ___scrt_acquire_startup_lock 1000d1e6 f   MSVCRT:utility.obj
 0001:0000c218       ___scrt_dllmain_after_initialize_c 1000d218 f   MSVCRT:utility.obj
 0001:0000c243       ___scrt_dllmain_before_initialize_c 1000d243 f   MSVCRT:utility.obj
 0001:0000c251       ___scrt_dllmain_crt_thread_attach 1000d251 f   MSVCRT:utility.obj
 0001:0000c270       ___scrt_dllmain_crt_thread_detach 1000d270 f   MSVCRT:utility.obj
 0001:0000c27d       ___scrt_dllmain_exception_filter 1000d27d f   MSVCRT:utility.obj
 0001:0000c2b1       ___scrt_dllmain_uninitialize_c 1000d2b1 f   MSVCRT:utility.obj
 0001:0000c2d4       ___scrt_dllmain_uninitialize_critical 1000d2d4 f   MSVCRT:utility.obj
 0001:0000c2e1       ___scrt_initialize_crt     1000d2e1 f   MSVCRT:utility.obj
 0001:0000c31a       ___scrt_initialize_onexit_tables 1000d31a f   MSVCRT:utility.obj
 0001:0000c3a1       ___scrt_is_nonwritable_in_current_image 1000d3a1 f   MSVCRT:utility.obj
 0001:0000c435       ___scrt_release_startup_lock 1000d435 f   MSVCRT:utility.obj
 0001:0000c452       ___scrt_uninitialize_crt   1000d452 f   MSVCRT:utility.obj
 0001:0000c47a       ___scrt_get_dyn_tls_init_callback 1000d47a f   MSVCRT:dyn_tls_init.obj
 0001:0000c480       ___scrt_fastfail           1000d480 f   MSVCRT:utility_desktop.obj
 0001:0000c59b       __crt_debugger_hook        1000d59b f   MSVCRT:utility_desktop.obj
 0001:0000c5a3       __RTC_Initialize           1000d5a3 f   MSVCRT:initsect.obj
 0001:0000c5cf       __RTC_Terminate            1000d5cf f   MSVCRT:initsect.obj
 0001:0000c600       __SEH_prolog4              1000d600 f   MSVCRT:sehprolg4.obj
 0001:0000c645       __except_handler4          1000d645 f   MSVCRT:chandler4gs.obj
 0001:0000c674       ___isa_available_init      1000d674 f   MSVCRT:cpu_disp.obj
 0001:0000c848       __get_startup_argv_mode    1000d848 f   MSVCRT:argv_mode.obj
 0001:0000c84c       ___scrt_is_ucrt_dll_in_use 1000d84c f   MSVCRT:ucrt_detection.obj
 0001:0000c858       _strchr                    1000d858 f   vcruntime:VCRUNTIME140.dll
 0001:0000c85e       _strstr                    1000d85e f   vcruntime:VCRUNTIME140.dll
 0001:0000c864       _memset                    1000d864 f   vcruntime:VCRUNTIME140.dll
 0001:0000c86a       _memcpy                    1000d86a f   vcruntime:VCRUNTIME140.dll
 0001:0000c870       ___std_type_info_destroy_list 1000d870 f   vcruntime:VCRUNTIME140.dll
 0001:0000c876       __except_handler4_common   1000d876 f   vcruntime:VCRUNTIME140.dll
 0001:0000c87c       _strcmp                    1000d87c f   ucrt:api-ms-win-crt-string-l1-1-0.dll
 0001:0000c882       _strlen                    1000d882 f   ucrt:api-ms-win-crt-string-l1-1-0.dll
 0001:0000c888       _strcpy                    1000d888 f   ucrt:api-ms-win-crt-string-l1-1-0.dll
 0001:0000c88e       _strcat                    1000d88e f   ucrt:api-ms-win-crt-string-l1-1-0.dll
 0001:0000c894       __initterm                 1000d894 f   ucrt:api-ms-win-crt-runtime-l1-1-0.dll
 0001:0000c89a       __initterm_e               1000d89a f   ucrt:api-ms-win-crt-runtime-l1-1-0.dll
 0001:0000c8a0       __seh_filter_dll           1000d8a0 f   ucrt:api-ms-win-crt-runtime-l1-1-0.dll
 0001:0000c8a6       __configure_narrow_argv    1000d8a6 f   ucrt:api-ms-win-crt-runtime-l1-1-0.dll
 0001:0000c8ac       __initialize_narrow_environment 1000d8ac f   ucrt:api-ms-win-crt-runtime-l1-1-0.dll
 0001:0000c8b2       __initialize_onexit_table  1000d8b2 f   ucrt:api-ms-win-crt-runtime-l1-1-0.dll
 0001:0000c8b8       __execute_onexit_table     1000d8b8 f   ucrt:api-ms-win-crt-runtime-l1-1-0.dll
 0001:0000c8be       __cexit                    1000d8be f   ucrt:api-ms-win-crt-runtime-l1-1-0.dll
 0001:0000c8c4       ___acrt_initialize         1000d8c4 f   MSVCRT:ucrt_stubs.obj
 0001:0000c8c4       ___acrt_thread_attach      1000d8c4 f   MSVCRT:ucrt_stubs.obj
 0001:0000c8c4       ___acrt_thread_detach      1000d8c4 f   MSVCRT:ucrt_stubs.obj
 0001:0000c8c4       ___acrt_uninitialize       1000d8c4 f   MSVCRT:ucrt_stubs.obj
 0001:0000c8c4       ___acrt_uninitialize_critical 1000d8c4 f   MSVCRT:ucrt_stubs.obj
 0001:0000c8c4       ___scrt_stub_for_acrt_initialize 1000d8c4 f   MSVCRT:ucrt_stubs.obj
 0001:0000c8c4       ___scrt_stub_for_acrt_thread_attach 1000d8c4 f   MSVCRT:ucrt_stubs.obj
 0001:0000c8c4       ___scrt_stub_for_acrt_thread_detach 1000d8c4 f   MSVCRT:ucrt_stubs.obj
 0001:0000c8c4       ___scrt_stub_for_acrt_uninitialize 1000d8c4 f   MSVCRT:ucrt_stubs.obj
 0001:0000c8c4       ___scrt_stub_for_acrt_uninitialize_critical 1000d8c4 f   MSVCRT:ucrt_stubs.obj
 0001:0000c8c4       ___vcrt_initialize         1000d8c4 f   MSVCRT:ucrt_stubs.obj
 0001:0000c8c4       ___vcrt_thread_attach      1000d8c4 f   MSVCRT:ucrt_stubs.obj
 0001:0000c8c4       ___vcrt_thread_detach      1000d8c4 f   MSVCRT:ucrt_stubs.obj
 0001:0000c8c4       ___vcrt_uninitialize       1000d8c4 f   MSVCRT:ucrt_stubs.obj
 0001:0000c8c4       ___vcrt_uninitialize_critical 1000d8c4 f   MSVCRT:ucrt_stubs.obj
 0001:0000c8c7       ___scrt_stub_for_is_c_termination_complete 1000d8c7 f   MSVCRT:ucrt_stubs.obj
 0001:0000c8c7       __is_c_termination_complete 1000d8c7 f   MSVCRT:ucrt_stubs.obj
 0001:0000c8ca       __filter_x86_sse2_floating_point_exception 1000d8ca f   MSVCRT:x86_exception_filter.obj
 0001:0000c8ca       __filter_x86_sse2_floating_point_exception_default 1000d8ca f   MSVCRT:x86_exception_filter.obj
 0002:00000000       __imp__RegCloseKey@4       1000e000     advapi32:ADVAPI32.dll
 0002:00000004       __imp__RegQueryValueExA@24 1000e004     advapi32:ADVAPI32.dll
 0002:00000008       __imp__RegOpenKeyExA@20    1000e008     advapi32:ADVAPI32.dll
 0002:0000000c       \177ADVAPI32_NULL_THUNK_DATA 1000e00c     advapi32:ADVAPI32.dll
 0002:00000010       __imp__SetUnhandledExceptionFilter@4 1000e010     kernel32:KERNEL32.dll
 0002:00000014       __imp__UnhandledExceptionFilter@4 1000e014     kernel32:KERNEL32.dll
 0002:00000018       __imp__LoadLibraryExA@12   1000e018     kernel32:KERNEL32.dll
 0002:0000001c       __imp__GetModuleHandleW@4  1000e01c     kernel32:KERNEL32.dll
 0002:00000020       __imp__FreeLibrary@4       1000e020     kernel32:KERNEL32.dll
 0002:00000024       __imp__VirtualQuery@12     1000e024     kernel32:KERNEL32.dll
 0002:00000028       __imp__VirtualProtect@16   1000e028     kernel32:KERNEL32.dll
 0002:0000002c       __imp__GetSystemInfo@4     1000e02c     kernel32:KERNEL32.dll
 0002:00000030       __imp__GetLastError@0      1000e030     kernel32:KERNEL32.dll
 0002:00000034       __imp__RaiseException@16   1000e034     kernel32:KERNEL32.dll
 0002:00000038       __imp__TerminateProcess@8  1000e038     kernel32:KERNEL32.dll
 0002:0000003c       __imp__EnterCriticalSection@4 1000e03c     kernel32:KERNEL32.dll
 0002:00000040       __imp__InitializeCriticalSection@4 1000e040     kernel32:KERNEL32.dll
 0002:00000044       __imp__GetOverlappedResult@16 1000e044     kernel32:KERNEL32.dll
 0002:00000048       __imp__MultiByteToWideChar@24 1000e048     kernel32:KERNEL32.dll
 0002:0000004c       __imp__GetProcAddress@8    1000e04c     kernel32:KERNEL32.dll
 0002:00000050       __imp__VerifyVersionInfoW@16 1000e050     kernel32:KERNEL32.dll
 0002:00000054       __imp__FormatMessageA@28   1000e054     kernel32:KERNEL32.dll
 0002:00000058       __imp__LocalFree@4         1000e058     kernel32:KERNEL32.dll
 0002:0000005c       __imp__VerSetConditionMask@16 1000e05c     kernel32:KERNEL32.dll
 0002:00000060       __imp__Sleep@4             1000e060     kernel32:KERNEL32.dll
 0002:00000064       __imp__SetHandleInformation@12 1000e064     kernel32:KERNEL32.dll
 0002:00000068       __imp__GetCurrentProcess@0 1000e068     kernel32:KERNEL32.dll
 0002:0000006c       __imp__IsProcessorFeaturePresent@4 1000e06c     kernel32:KERNEL32.dll
 0002:00000070       __imp__GetVersionExA@4     1000e070     kernel32:KERNEL32.dll
 0002:00000074       __imp__LeaveCriticalSection@4 1000e074     kernel32:KERNEL32.dll
 0002:00000078       __imp__GetCurrentProcessId@0 1000e078     kernel32:KERNEL32.dll
 0002:0000007c       __imp__GetCurrentThreadId@0 1000e07c     kernel32:KERNEL32.dll
 0002:00000080       __imp__GetSystemTimeAsFileTime@4 1000e080     kernel32:KERNEL32.dll
 0002:00000084       __imp__InitializeSListHead@4 1000e084     kernel32:KERNEL32.dll
 0002:00000088       __imp__IsDebuggerPresent@0 1000e088     kernel32:KERNEL32.dll
 0002:0000008c       __imp__QueryPerformanceCounter@4 1000e08c     kernel32:KERNEL32.dll
 0002:00000090       \177KERNEL32_NULL_THUNK_DATA 1000e090     kernel32:KERNEL32.dll
 0002:00000094       __imp___except_handler4_common 1000e094     vcruntime:VCRUNTIME140.dll
 0002:00000098       __imp____std_type_info_destroy_list 1000e098     vcruntime:VCRUNTIME140.dll
 0002:0000009c       __imp__memcpy              1000e09c     vcruntime:VCRUNTIME140.dll
 0002:000000a0       __imp__memset              1000e0a0     vcruntime:VCRUNTIME140.dll
 0002:000000a4       __imp__strstr              1000e0a4     vcruntime:VCRUNTIME140.dll
 0002:000000a8       __imp__strchr              1000e0a8     vcruntime:VCRUNTIME140.dll
 0002:000000ac       \177VCRUNTIME140_NULL_THUNK_DATA 1000e0ac     vcruntime:VCRUNTIME140.dll
 0002:000000b0       __imp__WSACleanup@0        1000e0b0     ws2_32:WS2_32.dll
 0002:000000b4       __imp__WSAStartup@8        1000e0b4     ws2_32:WS2_32.dll
 0002:000000b8       __imp__getprotobyname@4    1000e0b8     ws2_32:WS2_32.dll
 0002:000000bc       __imp__recv@16             1000e0bc     ws2_32:WS2_32.dll
 0002:000000c0       __imp__getnameinfo@28      1000e0c0     ws2_32:WS2_32.dll
 0002:000000c4       __imp__freeaddrinfo@4      1000e0c4     ws2_32:WS2_32.dll
 0002:000000c8       __imp__getaddrinfo@16      1000e0c8     ws2_32:WS2_32.dll
 0002:000000cc       __imp__WSAEventSelect@12   1000e0cc     ws2_32:WS2_32.dll
 0002:000000d0       __imp__WSACreateEvent@0    1000e0d0     ws2_32:WS2_32.dll
 0002:000000d4       __imp__WSACloseEvent@4     1000e0d4     ws2_32:WS2_32.dll
 0002:000000d8       __imp__gethostname@8       1000e0d8     ws2_32:WS2_32.dll
 0002:000000dc       __imp__gethostbyname@4     1000e0dc     ws2_32:WS2_32.dll
 0002:000000e0       __imp__gethostbyaddr@12    1000e0e0     ws2_32:WS2_32.dll
 0002:000000e4       __imp__WSASendDisconnect@8 1000e0e4     ws2_32:WS2_32.dll
 0002:000000e8       __imp__htons@4             1000e0e8     ws2_32:WS2_32.dll
 0002:000000ec       __imp__htonl@4             1000e0ec     ws2_32:WS2_32.dll
 0002:000000f0       __imp__getsockopt@20       1000e0f0     ws2_32:WS2_32.dll
 0002:000000f4       __imp__bind@12             1000e0f4     ws2_32:WS2_32.dll
 0002:000000f8       __imp__shutdown@8          1000e0f8     ws2_32:WS2_32.dll
 0002:000000fc       __imp__send@16             1000e0fc     ws2_32:WS2_32.dll
 0002:00000100       __imp__listen@8            1000e100     ws2_32:WS2_32.dll
 0002:00000104       __imp__closesocket@4       1000e104     ws2_32:WS2_32.dll
 0002:00000108       __imp__accept@12           1000e108     ws2_32:WS2_32.dll
 0002:0000010c       __imp____WSAFDIsSet@8      1000e10c     ws2_32:WS2_32.dll
 0002:00000110       __imp__WSAIoctl@36         1000e110     ws2_32:WS2_32.dll
 0002:00000114       __imp__WSAGetLastError@0   1000e114     ws2_32:WS2_32.dll
 0002:00000118       __imp__WSASetLastError@4   1000e118     ws2_32:WS2_32.dll
 0002:0000011c       __imp__socket@12           1000e11c     ws2_32:WS2_32.dll
 0002:00000120       __imp__setsockopt@20       1000e120     ws2_32:WS2_32.dll
 0002:00000124       __imp__sendto@24           1000e124     ws2_32:WS2_32.dll
 0002:00000128       __imp__select@20           1000e128     ws2_32:WS2_32.dll
 0002:0000012c       __imp__recvfrom@24         1000e12c     ws2_32:WS2_32.dll
 0002:00000130       __imp__ntohs@4             1000e130     ws2_32:WS2_32.dll
 0002:00000134       __imp__getsockname@12      1000e134     ws2_32:WS2_32.dll
 0002:00000138       __imp__ioctlsocket@12      1000e138     ws2_32:WS2_32.dll
 0002:0000013c       __imp__connect@12          1000e13c     ws2_32:WS2_32.dll
 0002:00000140       __imp__ntohl@4             1000e140     ws2_32:WS2_32.dll
 0002:00000144       \177WS2_32_NULL_THUNK_DATA 1000e144     ws2_32:WS2_32.dll
 0002:00000148       __imp__realloc             1000e148     ucrt:api-ms-win-crt-heap-l1-1-0.dll
 0002:0000014c       __imp__calloc              1000e14c     ucrt:api-ms-win-crt-heap-l1-1-0.dll
 0002:00000150       __imp__free                1000e150     ucrt:api-ms-win-crt-heap-l1-1-0.dll
 0002:00000154       __imp__malloc              1000e154     ucrt:api-ms-win-crt-heap-l1-1-0.dll
 0002:00000158       \177api-ms-win-crt-heap-l1-1-0_NULL_THUNK_DATA 1000e158     ucrt:api-ms-win-crt-heap-l1-1-0.dll
 0002:0000015c       __imp___execute_onexit_table 1000e15c     ucrt:api-ms-win-crt-runtime-l1-1-0.dll
 0002:00000160       __imp___cexit              1000e160     ucrt:api-ms-win-crt-runtime-l1-1-0.dll
 0002:00000164       __imp___initialize_narrow_environment 1000e164     ucrt:api-ms-win-crt-runtime-l1-1-0.dll
 0002:00000168       __imp___configure_narrow_argv 1000e168     ucrt:api-ms-win-crt-runtime-l1-1-0.dll
 0002:0000016c       __imp___seh_filter_dll     1000e16c     ucrt:api-ms-win-crt-runtime-l1-1-0.dll
 0002:00000170       __imp___initterm_e         1000e170     ucrt:api-ms-win-crt-runtime-l1-1-0.dll
 0002:00000174       __imp___initterm           1000e174     ucrt:api-ms-win-crt-runtime-l1-1-0.dll
 0002:00000178       __imp___initialize_onexit_table 1000e178     ucrt:api-ms-win-crt-runtime-l1-1-0.dll
 0002:0000017c       __imp___errno              1000e17c     ucrt:api-ms-win-crt-runtime-l1-1-0.dll
 0002:00000180       \177api-ms-win-crt-runtime-l1-1-0_NULL_THUNK_DATA 1000e180     ucrt:api-ms-win-crt-runtime-l1-1-0.dll
 0002:00000184       __imp____stdio_common_vfprintf 1000e184     ucrt:api-ms-win-crt-stdio-l1-1-0.dll
 0002:00000188       __imp____stdio_common_vsprintf 1000e188     ucrt:api-ms-win-crt-stdio-l1-1-0.dll
 0002:0000018c       __imp____stdio_common_vsscanf 1000e18c     ucrt:api-ms-win-crt-stdio-l1-1-0.dll
 0002:00000190       __imp____acrt_iob_func     1000e190     ucrt:api-ms-win-crt-stdio-l1-1-0.dll
 0002:00000194       __imp____stdio_common_vsnprintf_s 1000e194     ucrt:api-ms-win-crt-stdio-l1-1-0.dll
 0002:00000198       \177api-ms-win-crt-stdio-l1-1-0_NULL_THUNK_DATA 1000e198     ucrt:api-ms-win-crt-stdio-l1-1-0.dll
 0002:0000019c       __imp__isspace             1000e19c     ucrt:api-ms-win-crt-string-l1-1-0.dll
 0002:000001a0       __imp__strcpy              1000e1a0     ucrt:api-ms-win-crt-string-l1-1-0.dll
 0002:000001a4       __imp__strlen              1000e1a4     ucrt:api-ms-win-crt-string-l1-1-0.dll
 0002:000001a8       __imp__strtok_s            1000e1a8     ucrt:api-ms-win-crt-string-l1-1-0.dll
 0002:000001ac       __imp__strncmp             1000e1ac     ucrt:api-ms-win-crt-string-l1-1-0.dll
 0002:000001b0       __imp__wcslen              1000e1b0     ucrt:api-ms-win-crt-string-l1-1-0.dll
 0002:000001b4       __imp__strncpy_s           1000e1b4     ucrt:api-ms-win-crt-string-l1-1-0.dll
 0002:000001b8       __imp__strncpy             1000e1b8     ucrt:api-ms-win-crt-string-l1-1-0.dll
 0002:000001bc       __imp__strcmp              1000e1bc     ucrt:api-ms-win-crt-string-l1-1-0.dll
 0002:000001c0       __imp__wcscpy              1000e1c0     ucrt:api-ms-win-crt-string-l1-1-0.dll
 0002:000001c4       __imp__strcat              1000e1c4     ucrt:api-ms-win-crt-string-l1-1-0.dll
 0002:000001c8       \177api-ms-win-crt-string-l1-1-0_NULL_THUNK_DATA 1000e1c8     ucrt:api-ms-win-crt-string-l1-1-0.dll
 0002:000001cc       __imp__getErrorString      1000e1cc     java:java.dll
 0002:000001d0       __imp__JNU_ThrowByNameWithMessageAndLastError@12 1000e1d0     java:java.dll
 0002:000001d4       __imp__JNU_NewStringPlatform@8 1000e1d4     java:java.dll
 0002:000001d8       __imp__JNU_ThrowOutOfMemoryError@8 1000e1d8     java:java.dll
 0002:000001dc       __imp__JNU_ThrowByName@12  1000e1dc     java:java.dll
 0002:000001e0       __imp__JNU_ThrowByNameWithLastError@12 1000e1e0     java:java.dll
 0002:000001e4       __imp__JNU_ThrowNullPointerException@8 1000e1e4     java:java.dll
 0002:000001e8       __imp__JNU_ReleaseStringPlatformChars@12 1000e1e8     java:java.dll
 0002:000001ec       __imp__JNU_GetStringPlatformChars@12 1000e1ec     java:java.dll
 0002:000001f0       __imp__JDK_LoadSystemLibrary 1000e1f0     java:java.dll
 0002:000001f4       \177java_NULL_THUNK_DATA   1000e1f4     java:java.dll
 0002:000001f8       __imp__jio_snprintf        1000e1f8     jvm:jvm.dll
 0002:000001fc       __imp__JVM_InitializeSocketLibrary@0 1000e1fc     jvm:jvm.dll
 0002:00000200       __imp__JVM_CurrentTimeMillis@8 1000e200     jvm:jvm.dll
 0002:00000204       \177jvm_NULL_THUNK_DATA    1000e204     jvm:jvm.dll
 0002:00000208       ___guard_check_icall_fptr  1000e208     MSVCRT:guard_support.obj
 0002:0000020c       ___castguard_check_failure_os_handled_fptr 1000e20c     MSVCRT:guard_support.obj
 0002:00000210       ___xc_a                    1000e210     MSVCRT:initializers.obj
 0002:00000214       ___xc_z                    1000e214     MSVCRT:initializers.obj
 0002:00000218       ___xi_a                    1000e218     MSVCRT:initializers.obj
 0002:0000021c       ___xi_z                    1000e21c     MSVCRT:initializers.obj
 0002:00000220       ___xp_a                    1000e220     MSVCRT:initializers.obj
 0002:00000224       ___xp_z                    1000e224     MSVCRT:initializers.obj
 0002:00000228       ___xt_a                    1000e228     MSVCRT:initializers.obj
 0002:0000022c       ___xt_z                    1000e22c     MSVCRT:initializers.obj
 0002:00000230       ??_C@_0BH@FIKCFBLO@Ljava?1net?1InetAddress?$DL@ 1000e230     DatagramPacket.obj
 0002:00000248       ??_C@_07LHEPONKL@address@  1000e248     DatagramPacket.obj
 0002:00000250       ??_C@_01JPJNBJEM@I@        1000e250     DatagramPacket.obj
 0002:00000254       ??_C@_04LPGMAPLE@port@     1000e254     DatagramPacket.obj
 0002:0000025c       ??_C@_02KCBIMKDL@?$FLB@    1000e25c     DatagramPacket.obj
 0002:00000260       ??_C@_03COAJHJPB@buf@      1000e260     DatagramPacket.obj
 0002:00000264       ??_C@_06KLHHMIGM@offset@   1000e264     DatagramPacket.obj
 0002:0000026c       ??_C@_06IJDLPEM@length@    1000e26c     DatagramPacket.obj
 0002:00000274       ??_C@_09MAGKMKDD@bufLength@ 1000e274     DatagramPacket.obj
 0002:00000280       ??_C@_0P@CALONDPA@java?1net?1Proxy@ 1000e280     DefaultProxySelector.obj
 0002:00000290       ??_C@_0BH@EIEAJJDI@JNI?5errror?5at?5line?5?$CFd?6@ 1000e290     DefaultProxySelector.obj
 0002:000002a8       ??_C@_0BE@CNHDIHBN@java?1net?1Proxy$Type@ 1000e2a8     DefaultProxySelector.obj
 0002:000002bc       ??_C@_0BL@HBNNAPLM@java?1net?1InetSocketAddress@ 1000e2bc     DefaultProxySelector.obj
 0002:000002d8       ??_C@_0DB@PIODMB@?$CILjava?1net?1Proxy$Type?$DLLjava?1net@ 1000e2d8     DefaultProxySelector.obj
 0002:0000030c       ??_C@_06FALKBLGB@?$DMinit?$DO@ 1000e30c     DefaultProxySelector.obj
 0002:00000314       ??_C@_0BB@GMCFBELK@Ljava?1net?1Proxy?$DL@ 1000e314     DefaultProxySelector.obj
 0002:00000328       ??_C@_08KOHKDPPJ@NO_PROXY@ 1000e328     DefaultProxySelector.obj
 0002:00000334       ??_C@_0BG@JJBIBCMK@Ljava?1net?1Proxy$Type?$DL@ 1000e334     DefaultProxySelector.obj
 0002:0000034c       ??_C@_04MEDPFIKH@HTTP@     1000e34c     DefaultProxySelector.obj
 0002:00000354       ??_C@_05HKHMHAPI@SOCKS@    1000e354     DefaultProxySelector.obj
 0002:0000035c       ??_C@_0DC@FDHLAKNF@?$CILjava?1lang?1String?$DLI?$CJLjava?1net?1@ 1000e35c     DefaultProxySelector.obj
 0002:00000390       ??_C@_0BB@BNNOLJPL@createUnresolved@ 1000e390     DefaultProxySelector.obj
 0002:000003a4       ??_C@_0DM@IMMDCFC@Software?2Microsoft?2Windows?2Curr@ 1000e3a4     DefaultProxySelector.obj
 0002:000003e0       ??_C@_0M@IOGAMEAC@ProxyEnable@ 1000e3e0     DefaultProxySelector.obj
 0002:000003ec       ??_C@_0O@KBIEAGIG@ProxyOverride@ 1000e3ec     DefaultProxySelector.obj
 0002:000003fc       ??_C@_0M@BCMAAPLG@ProxyServer@ 1000e3fc     DefaultProxySelector.obj
 0002:00000408       ??_C@_02LNAEAIDO@?$DL?5@   1000e408     DefaultProxySelector.obj
 0002:0000040c       ??_C@_04IAFLKNP@http@      1000e40c     DefaultProxySelector.obj
 0002:00000414       ??_C@_03LMDBDBEG@ftp@      1000e414     DefaultProxySelector.obj
 0002:00000418       ??_C@_06IBHFMCPJ@gopher@   1000e418     DefaultProxySelector.obj
 0002:00000420       ??_C@_05BCHGOAMK@https@    1000e420     DefaultProxySelector.obj
 0002:00000428       ??_C@_05LBOKJHLG@socks@    1000e428     DefaultProxySelector.obj
 0002:00000430       ??_C@_03HFAIOBFI@?$CFs?$DN@ 1000e430     DefaultProxySelector.obj
 0002:00000434       ??_C@_02DPKJAMEF@?$CFd@    1000e434     DefaultProxySelector.obj
 0002:00000438       ??_C@_0BJ@BDFOFHPL@Ljava?1io?1FileDescriptor?$DL@ 1000e438     DualStackPlainDatagramSocketImpl.obj
 0002:00000454       ??_C@_02ENHFDPNM@fd@       1000e454     DualStackPlainDatagramSocketImpl.obj
 0002:00000458       ??_C@_0BH@HIFKKJJA@Socket?5creation?5failed@ 1000e458     DualStackPlainDatagramSocketImpl.obj
 0002:00000470       ??_C@_0M@PJEGOMKJ@Cannot?5bind@ 1000e470     DualStackPlainDatagramSocketImpl.obj
 0002:0000047c       ??_C@_07KAIBNCHO@connect@  1000e47c     DualStackPlainDatagramSocketImpl.obj
 0002:00000484       ??_C@_0BA@IBCMDLCP@JVM_GetSockName@ 1000e484     DualStackPlainDatagramSocketImpl.obj
 0002:00000494       ??_C@_0BK@JGFJKHKC@Error?5getting?5socket?5name@ 1000e494     DualStackPlainDatagramSocketImpl.obj
 0002:000004b0       ??_C@_0BO@IKFIAFAI@Native?5heap?5allocation?5failed@ 1000e4b0     DualStackPlainDatagramSocketImpl.obj
 0002:000004d0       ??_C@_0BC@FEBIBOEI@Receive?5timed?5out@ 1000e4d0     DualStackPlainDatagramSocketImpl.obj
 0002:000004e4       ??_C@_0CA@FIMHICIJ@java?1net?1SocketTimeoutException@ 1000e4e4     DualStackPlainDatagramSocketImpl.obj
 0002:00000504       ??_C@_0O@PLGOCGPF@Socket?5closed@ 1000e504     DualStackPlainDatagramSocketImpl.obj
 0002:00000514       ??_C@_0BJ@IJNLNPKI@java?1net?1SocketException@ 1000e514     DualStackPlainDatagramSocketImpl.obj
 0002:00000530       ??_C@_0BG@DCFFKIHC@operation?5interrupted@ 1000e530     DualStackPlainDatagramSocketImpl.obj
 0002:00000548       ??_C@_0BP@DENMAKHD@java?1io?1InterruptedIOException@ 1000e548     DualStackPlainDatagramSocketImpl.obj
 0002:00000568       ??_C@_0BG@EDMCJFNE@ICMP?5Port?5Unreachable@ 1000e568     DualStackPlainDatagramSocketImpl.obj
 0002:00000580       ??_C@_0CC@BDDMPFBF@java?1net?1PortUnreachableExcepti@ 1000e580     DualStackPlainDatagramSocketImpl.obj
 0002:000005a4       ??_C@_0O@DGAKFOCN@socket?5closed@ 1000e5a4     DualStackPlainDatagramSocketImpl.obj
 0002:000005b4       ??_C@_0BI@GDLKKOMD@Datagram?5receive?5failed@ 1000e5b4     DualStackPlainDatagramSocketImpl.obj
 0002:000005cc       ??_C@_0BF@DHIDENDP@Datagram?5send?5failed@ 1000e5cc     DualStackPlainDatagramSocketImpl.obj
 0002:000005e4       ??_C@_0P@HBJFFFFJ@Invalid?5option@ 1000e5e4     DualStackPlainDatagramSocketImpl.obj
 0002:000005f4       ??_C@_0L@CKHNIFCM@setsockopt@ 1000e5f4     DualStackPlainDatagramSocketImpl.obj
 0002:00000600       ??_C@_0L@DEFCDCGF@getsockopt@ 1000e600     DualStackPlainDatagramSocketImpl.obj
 0002:0000060c       ??_C@_0BL@KCCEIBDI@?$CILjava?1net?1InetAddress?$DLI?$CJV@ 1000e60c     DualStackPlainSocketImpl.obj
 0002:00000628       ??_C@_06HBNONAG@create@    1000e628     DualStackPlainSocketImpl.obj
 0002:00000630       ??_C@_08DOMCMNDL@JVM_Bind@ 1000e630     DualStackPlainSocketImpl.obj
 0002:00000640       ??_C@_0FF@BAOCINGB@connect?3?5Address?5is?5invalid?5on?5@ 1000e640     DualStackPlainSocketImpl.obj
 0002:00000698       ??_C@_0BK@LKDLOIJL@java?1net?1ConnectException@ 1000e698     DualStackPlainSocketImpl.obj
 0002:000006b4       ??_C@_0BC@DJFNFCAI@connect?5timed?5out@ 1000e6b4     DualStackPlainSocketImpl.obj
 0002:000006c8       ??_C@_0BP@PANEALJE@Unable?5to?5establish?5connection@ 1000e6c8     DualStackPlainSocketImpl.obj
 0002:000006e8       ??_C@_0BD@PDGFKJCK@getsockname?5failed@ 1000e6e8     DualStackPlainSocketImpl.obj
 0002:000006fc       ??_C@_04HLBMEOMD@addr@     1000e6fc     DualStackPlainSocketImpl.obj
 0002:00000704       ??_C@_0O@MHKNJCGE@listen?5failed@ 1000e704     DualStackPlainSocketImpl.obj
 0002:00000714       ??_C@_0BB@JOKEJOH@Accept?5timed?5out@ 1000e714     DualStackPlainSocketImpl.obj
 0002:00000728       ??_C@_0BB@DIMAMJLH@socket?5available@ 1000e728     DualStackPlainSocketImpl.obj
 0002:0000073c       ??_C@_0BK@BFOOMAAO@Unsupported?5socket?5option@ 1000e73c     DualStackPlainSocketImpl.obj
 0002:00000758       ??_C@_04MIIPNNEF@send@     1000e758     DualStackPlainSocketImpl.obj
 0002:00000760       ??_C@_0BC@GBCMOPPJ@configureBlocking@ 1000e760     DualStackPlainSocketImpl.obj
 0002:00000774       ??_C@_0BK@JKDLHALP@unsupported?5socket?5option@ 1000e774     ExtendedOptionsImpl.obj
 0002:00000790       ??_C@_0CI@LDDEGNGM@java?1lang?1UnsupportedOperationE@ 1000e790     ExtendedOptionsImpl.obj
 0002:000007b8       ??_C@_0BG@MGDLLCGN@java?1net?1Inet4Address@ 1000e7b8     Inet4Address.obj
 0002:000007d0       ??_C@_03GAEACAIP@?$CI?$CJV@ 1000e7d0     Inet4Address.obj
 0002:000007d4       ??_C@_09IPAEKDAI@localhost@ 1000e7d4     Inet4AddressImpl.obj
 0002:000007e0       ??_C@_0O@DOOCGKOP@host?5argument@ 1000e7e0     Inet4AddressImpl.obj
 0002:000007f0       ??_C@_0BO@JEDADEEB@java?1net?1UnknownHostException@ 1000e7f0     Inet4AddressImpl.obj
 0002:00000810       ??_C@_0BE@KNBHMLLP@Can?8t?5create?5socket@ 1000e810     Inet4AddressImpl.obj
 0002:00000824       ??_C@_0BC@LNOJFPHG@Can?8t?5bind?5socket@ 1000e824     Inet4AddressImpl.obj
 0002:00000838       ??_C@_0P@FKKLKLOM@connect?5failed@ 1000e838     Inet4AddressImpl.obj
 0002:00000848       ??_C@_0BK@CJOLIFJC@Unable?5to?5allocate?5memory@ 1000e848     Inet4AddressImpl.obj
 0002:00000864       ??_C@_0CC@EAIDNHEI@Unable?5to?5create?5ICMP?5file?5hand@ 1000e864     Inet4AddressImpl.obj
 0002:00000888       ??_C@_0BG@OIMNJKOL@java?1net?1Inet6Address@ 1000e888     Inet6Address.obj
 0002:000008a0       ??_C@_0CJ@HANKHEO@java?1net?1Inet6Address$Inet6Addr@ 1000e8a0     Inet6Address.obj
 0002:000008cc       ??_C@_0CL@OGPDIPGP@Ljava?1net?1Inet6Address$Inet6Add@ 1000e8cc     Inet6Address.obj
 0002:000008f8       ??_C@_07CFDIJDEC@holder6@  1000e8f8     Inet6Address.obj
 0002:00000900       ??_C@_09OMLGLGNL@ipaddress@ 1000e900     Inet6Address.obj
 0002:0000090c       ??_C@_08HMELDLBB@scope_id@ 1000e90c     Inet6Address.obj
 0002:00000918       ??_C@_0BA@CBBKEDDC@cached_scope_id@ 1000e918     Inet6Address.obj
 0002:00000928       ??_C@_01POHCFINO@Z@        1000e928     Inet6Address.obj
 0002:0000092c       ??_C@_0N@EMCDHDAD@scope_id_set@ 1000e92c     Inet6Address.obj
 0002:0000093c       ??_C@_0BM@MEIIMOAC@Ljava?1net?1NetworkInterface?$DL@ 1000e93c     Inet6Address.obj
 0002:00000958       ??_C@_0N@DKHAKOIC@scope_ifname@ 1000e958     Inet6Address.obj
 0002:00000968       ??_C@_0N@DMACLPJ@host?5is?5null@ 1000e968     Inet6AddressImpl.obj
 0002:00000978       ??_C@_0BP@NBCDDEJF@Can?8t?5bind?5socket?5to?5interface@ 1000e978     Inet6AddressImpl.obj
 0002:00000998       ??_C@_0BF@LNJHKELF@java?1net?1InetAddress@ 1000e998     InetAddress.obj
 0002:000009b0       ??_C@_0CH@OBMJDEDM@java?1net?1InetAddress$InetAddres@ 1000e9b0     InetAddress.obj
 0002:000009d8       ??_C@_0CJ@BPCMNDLL@Ljava?1net?1InetAddress$InetAddre@ 1000e9d8     InetAddress.obj
 0002:00000a04       ??_C@_06JIPLHHCL@holder@   1000ea04     InetAddress.obj
 0002:00000a0c       ??_C@_0BC@LHOCKAOM@preferIPv6Address@ 1000ea0c     InetAddress.obj
 0002:00000a20       ??_C@_06NBOBHOCP@family@   1000ea20     InetAddress.obj
 0002:00000a28       ??_C@_0BD@JFADHEFE@Ljava?1lang?1String?$DL@ 1000ea28     InetAddress.obj
 0002:00000a3c       ??_C@_08IGGJEOEE@hostName@ 1000ea3c     InetAddress.obj
 0002:00000a48       ??_C@_0BB@JAHGOJG@originalHostName@ 1000ea48     InetAddress.obj
 0002:00000a5c       ??_C@_01LELAEKIP@J@        1000ea5c     NTLMAuthSequence.obj
 0002:00000a60       ??_C@_09ILBCNDDJ@ctxHandle@ 1000ea60     NTLMAuthSequence.obj
 0002:00000a6c       ??_C@_09NDBMIONH@crdHandle@ 1000ea6c     NTLMAuthSequence.obj
 0002:00000a78       ??_C@_0BB@KLNFJBDM@sequenceComplete@ 1000ea78     NTLMAuthSequence.obj
 0002:00000a8c       ??_C@_0CA@NIIGFDJD@native?5memory?5allocation?5failed@ 1000ea8c     NTLMAuthSequence.obj
 0002:00000aac       ??_C@_04KGCGDDND@NTLM@     1000eaac     NTLMAuthSequence.obj
 0002:00000ab4       ??_C@_0L@BFDIJHCF@urlmon?4dll@ 1000eab4     NTLMAuthentication.obj
 0002:00000ac0       ??_C@_0CA@OOMLPODH@CoInternetCreateSecurityManager@ 1000eac0     NTLMAuthentication.obj
 0002:00000ae0       ??_C@_0BP@FOGJMHII@Native?5heap?5allocation?5failure@ 1000eae0     NetworkInterface.obj
 0002:00000b00       ??_C@_0CN@IHAKACDK@IP?5Helper?5Library?5GetIfTable?5fu@ 1000eb00     NetworkInterface.obj
 0002:00000b30       ??_C@_0BA@NOLMKEPF@java?1lang?1Error@ 1000eb30     NetworkInterface.obj
 0002:00000b40       ??_C@_05NLNDHDPO@eth?$CFd@ 1000eb40     NetworkInterface.obj
 0002:00000b48       ??_C@_04MLKOAMFC@tr?$CFd@  1000eb48     NetworkInterface.obj
 0002:00000b50       ??_C@_06MBLFHLO@fddi?$CFd@ 1000eb50     NetworkInterface.obj
 0002:00000b58       ??_C@_02KDBGGDMB@lo@       1000eb58     NetworkInterface.obj
 0002:00000b5c       ??_C@_05OIOFDJGG@ppp?$CFd@ 1000eb5c     NetworkInterface.obj
 0002:00000b64       ??_C@_04MJEIPAOO@sl?$CFd@  1000eb64     NetworkInterface.obj
 0002:00000b6c       ??_C@_06HENGPFGA@wlan?$CFd@ 1000eb6c     NetworkInterface.obj
 0002:00000b74       ??_C@_05PGFLNFCI@net?$CFd@ 1000eb74     NetworkInterface.obj
 0002:00000b7c       ??_C@_0DF@NKGEGFCE@Cannot?5get?5multibyte?5char?5for?5i@ 1000eb7c     NetworkInterface.obj
 0002:00000bb4       ??_C@_0DB@GGBHCAPL@IP?5Helper?5Library?5GetIpAddrTabl@ 1000ebb4     NetworkInterface.obj
 0002:00000be8       ??_C@_04MEMAJGDJ@name@     1000ebe8     NetworkInterface.obj
 0002:00000bf0       ??_C@_0M@NDEOCEGH@displayName@ 1000ebf0     NetworkInterface.obj
 0002:00000bfc       ??_C@_05FKHKFDID@index@    1000ebfc     NetworkInterface.obj
 0002:00000c04       ??_C@_0BI@FKGHKPME@?$FLLjava?1net?1InetAddress?$DL@ 1000ec04     NetworkInterface.obj
 0002:00000c1c       ??_C@_05GAEKFHB@addrs@     1000ec1c     NetworkInterface.obj
 0002:00000c24       ??_C@_0BN@FGCEFHCI@?$FLLjava?1net?1InterfaceAddress?$DL@ 1000ec24     NetworkInterface.obj
 0002:00000c44       ??_C@_08OKHKOBIL@bindings@ 1000ec44     NetworkInterface.obj
 0002:00000c50       ??_C@_0BN@LEABGBNB@?$FLLjava?1net?1NetworkInterface?$DL@ 1000ec50     NetworkInterface.obj
 0002:00000c70       ??_C@_06JCHEOPIA@childs@   1000ec70     NetworkInterface.obj
 0002:00000c78       ??_C@_0BK@HBDFEEEP@java?1net?1InterfaceAddress@ 1000ec78     NetworkInterface.obj
 0002:00000c94       ??_C@_0BI@EDMBHPFP@Ljava?1net?1Inet4Address?$DL@ 1000ec94     NetworkInterface.obj
 0002:00000cac       ??_C@_09OALBOHJN@broadcast@ 1000ecac     NetworkInterface.obj
 0002:00000cb8       ??_C@_01CPLAODJH@S@        1000ecb8     NetworkInterface.obj
 0002:00000cbc       ??_C@_0L@NAAPBPMO@maskLength@ 1000ecbc     NetworkInterface.obj
 0002:00000cc8       _BUFF_SIZE                 1000ecc8     NetworkInterface_winXP.obj
 0002:00000ccc       _MAX_TRIES                 1000eccc     NetworkInterface_winXP.obj
 0002:00000cd0       ??_C@_0BL@ENCPOIKC@java?1lang?1OutOfMemoryError@ 1000ecd0     NetworkInterface_winXP.obj
 0002:00000cec       ??_C@_0DH@HIDBKCBL@IP?5Helper?5Library?5GetAdaptersAd@ 1000ecec     NetworkInterface_winXP.obj
 0002:00000d24       ??_C@_05LFCNEKM@tun?$CFd@  1000ed24     NetworkInterface_winXP.obj
 0002:00000d2c       ??_C@_01CLKCMJKC@?5@       1000ed2c     ResolverConfigurationImpl.obj
 0002:00000d30       ??_C@_0DD@IKBMIFKO@SYSTEM?2CurrentControlSet?2Servic@ 1000ed30     ResolverConfigurationImpl.obj
 0002:00000d64       ??_C@_0L@HPLHIFHN@SearchList@ 1000ed64     ResolverConfigurationImpl.obj
 0002:00000d70       ??_C@_0EB@FEBCMLKE@SYSTEM?2CurrentControlSet?2Servic@ 1000ed70     ResolverConfigurationImpl.obj
 0002:00000db4       ??_C@_0L@HPPGIMO@EnableDhcp@ 1000edb4     ResolverConfigurationImpl.obj
 0002:00000dc0       ??_C@_06HFDFFJHI@Domain@   1000edc0     ResolverConfigurationImpl.obj
 0002:00000dc8       ??_C@_0L@OOMBDFPC@DhcpDomain@ 1000edc8     ResolverConfigurationImpl.obj
 0002:00000dd4       ??_C@_0L@MPBDOIAL@NameServer@ 1000edd4     ResolverConfigurationImpl.obj
 0002:00000de0       ??_C@_0P@BLDHOCGF@DhcpNameServer@ 1000ede0     ResolverConfigurationImpl.obj
 0002:00000df0       ??_C@_0O@BBEOADGN@os_searchlist@ 1000edf0     ResolverConfigurationImpl.obj
 0002:00000e00       ??_C@_0P@HAAMGONH@os_nameservers@ 1000ee00     ResolverConfigurationImpl.obj
 0002:00000e10       ??_C@_0P@MNGKMEOF@Read?5timed?5out@ 1000ee10     SocketInputStream.obj
 0002:00000e20       ??_C@_0BG@LKMKDKLB@Operation?5interrupted@ 1000ee20     SocketInputStream.obj
 0002:00000e38       ??_C@_0O@DENDBPGJ@Socket?5Closed@ 1000ee38     SocketInputStream.obj
 0002:00000e46       ??_C@_00CNPNBAHC@@         1000ee46     SocketInputStream.obj
 0002:00000e48       ??_C@_0CB@LJKAIJOC@sun?1net?1ConnectionResetExceptio@ 1000ee48     SocketInputStream.obj
 0002:00000e6c       ??_C@_0M@KMFGCEDE@recv?5failed@ 1000ee6c     SocketInputStream.obj
 0002:00000e78       ??_C@_0O@EFMIHGHE@data?5argument@ 1000ee78     SocketOutputStream.obj
 0002:00000e88       ??_C@_0DP@KCKHLBJL@No?5buffer?5space?5available?5?9?5exh@ 1000ee88     SocketOutputStream.obj
 0002:00000ec8       ??_C@_0BD@PIDCCABF@socket?5write?5error@ 1000eec8     SocketOutputStream.obj
 0002:00000edc       ??_C@_0BC@OHJKABOO@java?1lang?1Integer@ 1000eedc     TwoStacksPlainDatagramSocketImpl.obj
 0002:00000ef0       ??_C@_04PFANPMCN@?$CII?$CJV@ 1000eef0     TwoStacksPlainDatagramSocketImpl.obj
 0002:00000ef8       ??_C@_0BC@DDPBLLCP@java?1lang?1Boolean@ 1000eef8     TwoStacksPlainDatagramSocketImpl.obj
 0002:00000f0c       ??_C@_04LHKBAEFM@?$CIZ?$CJV@ 1000ef0c     TwoStacksPlainDatagramSocketImpl.obj
 0002:00000f14       ??_C@_0BK@CKMMMKHL@Unable?5to?5obtain?5hostname@ 1000ef14     TwoStacksPlainDatagramSocketImpl.obj
 0002:00000f30       ??_C@_03EJHFOMHC@fd1@      1000ef30     TwoStacksPlainDatagramSocketImpl.obj
 0002:00000f34       ??_C@_07DDHNKDGP@timeout@  1000ef34     TwoStacksPlainDatagramSocketImpl.obj
 0002:00000f3c       ??_C@_05OOPOHKND@fduse@    1000ef3c     TwoStacksPlainDatagramSocketImpl.obj
 0002:00000f44       ??_C@_06PKMJGOAK@lastfd@   1000ef44     TwoStacksPlainDatagramSocketImpl.obj
 0002:00000f4c       ??_C@_0N@FBKGBGNJ@trafficClass@ 1000ef4c     TwoStacksPlainDatagramSocketImpl.obj
 0002:00000f5c       ??_C@_09BPJHDKHI@localPort@ 1000ef5c     TwoStacksPlainDatagramSocketImpl.obj
 0002:00000f68       ??_C@_09JGOMOAGJ@connected@ 1000ef68     TwoStacksPlainDatagramSocketImpl.obj
 0002:00000f74       ??_C@_0BH@MPHCPCAM@java?1io?1FileDescriptor@ 1000ef74     TwoStacksPlainDatagramSocketImpl.obj
 0002:00000f8c       ??_C@_0BO@EBCCBLCJ@Protocol?5family?5not?5supported@ 1000ef8c     TwoStacksPlainDatagramSocketImpl.obj
 0002:00000fac       ??_C@_0BB@IGCLOFNO@argument?5address@ 1000efac     TwoStacksPlainDatagramSocketImpl.obj
 0002:00000fc0       ??_C@_0M@FKPMEIFN@null?5packet@ 1000efc0     TwoStacksPlainDatagramSocketImpl.obj
 0002:00000fcc       ??_C@_0BM@DPDKEIHM@null?5address?5?$HM?$HM?5null?5buffer@ 1000efcc     TwoStacksPlainDatagramSocketImpl.obj
 0002:00000fe8       ??_C@_0BF@LKFFGFKN@Protocol?5not?5allowed@ 1000efe8     TwoStacksPlainDatagramSocketImpl.obj
 0002:00001000       ??_C@_0CH@HCKHFPHO@Send?5buf?5native?5heap?5allocation@ 1000f000     TwoStacksPlainDatagramSocketImpl.obj
 0002:00001028       ??_C@_0BH@OBJCPBFA@Null?5address?5in?5peek?$CI?$CJ@ 1000f028     TwoStacksPlainDatagramSocketImpl.obj
 0002:00001040       ??_C@_0P@NHMBIAJD@Peek?5timed?5out@ 1000f040     TwoStacksPlainDatagramSocketImpl.obj
 0002:00001050       ??_C@_0CA@LHJKECEL@timeout?5in?5datagram?5socket?5peek@ 1000f050     TwoStacksPlainDatagramSocketImpl.obj
 0002:00001070       ??_C@_0BF@GHEEKLOJ@Datagram?5peek?5failed@ 1000f070     TwoStacksPlainDatagramSocketImpl.obj
 0002:00001088       ??_C@_06HKKJOEPD@packet@   1000f088     TwoStacksPlainDatagramSocketImpl.obj
 0002:00001090       ??_C@_0O@EEGMFPKK@packet?5buffer@ 1000f090     TwoStacksPlainDatagramSocketImpl.obj
 0002:000010a0       ??_C@_0CK@LJPBFGBB@Receive?5buf?5native?5heap?5allocat@ 1000f0a0     TwoStacksPlainDatagramSocketImpl.obj
 0002:000010cc       ??_C@_0BK@OMHJKJIG@java?1net?1NetworkInterface@ 1000f0cc     TwoStacksPlainDatagramSocketImpl.obj
 0002:000010e8       ??_C@_0EG@BPIHIIBO@bad?5argument?5for?5IP_MULTICAST_I@ 1000f0e8     TwoStacksPlainDatagramSocketImpl.obj
 0002:00001130       ??_C@_0EF@JBMEFJAO@bad?5argument?5for?5IP_MULTICAST_I@ 1000f130     TwoStacksPlainDatagramSocketImpl.obj
 0002:00001178       ??_C@_0BM@NAPLPNMN@Error?5setting?5socket?5option@ 1000f178     TwoStacksPlainDatagramSocketImpl.obj
 0002:00001194       ??_C@_0DM@IFNIENGO@IPV6_MULTICAST_IF?5failed?5?$CIinter@ 1000f194     TwoStacksPlainDatagramSocketImpl.obj
 0002:000011d0       ??_C@_0CL@DOKPHAMI@no?5InetAddress?5instances?5of?5req@ 1000f1d0     TwoStacksPlainDatagramSocketImpl.obj
 0002:000011fc       ??_C@_05MFEJDJP@value@     1000f1fc     TwoStacksPlainDatagramSocketImpl.obj
 0002:00001204       ??_C@_0DG@HAOMPAGJ@Socket?5option?5not?5supported?5by?5@ 1000f204     TwoStacksPlainDatagramSocketImpl.obj
 0002:0000123c       ??_C@_0BA@KNNGAGBM@setsockopt?5IPv6@ 1000f23c     TwoStacksPlainDatagramSocketImpl.obj
 0002:0000124c       ??_C@_0BM@CFKNCEIM@Error?5getting?5socket?5option@ 1000f24c     TwoStacksPlainDatagramSocketImpl.obj
 0002:00001268       ??_C@_0BJ@PCBGABPN@?$CI?$CJLjava?1net?1InetAddress?$DL@ 1000f268     TwoStacksPlainDatagramSocketImpl.obj
 0002:00001284       ??_C@_0BA@ILEICAKK@anyLocalAddress@ 1000f284     TwoStacksPlainDatagramSocketImpl.obj
 0002:00001294       ??_C@_0DP@FFHJMIJA@IPV6_MULTICAST_IF?5returned?5inde@ 1000f294     TwoStacksPlainDatagramSocketImpl.obj
 0002:000012d4       ??_C@_0DJ@HEGBECIK@IPV6_MULTICAST_IF?5returned?5inte@ 1000f2d4     TwoStacksPlainDatagramSocketImpl.obj
 0002:00001310       ??_C@_0CA@IDODINKJ@error?5getting?5socket?5option?3?5?$CFs@ 1000f310     TwoStacksPlainDatagramSocketImpl.obj
 0002:00001330       ??_C@_0EA@FEALAIDB@Socket?5option?5not?5supported?5by?5@ 1000f330     TwoStacksPlainDatagramSocketImpl.obj
 0002:00001370       ??_C@_0BM@KFCLABAN@set?5IP_MULTICAST_TTL?5failed@ 1000f370     TwoStacksPlainDatagramSocketImpl.obj
 0002:0000138c       ??_C@_0BP@FKDKMPAN@set?5IPV6_MULTICAST_HOPS?5failed@ 1000f38c     TwoStacksPlainDatagramSocketImpl.obj
 0002:000013ac       ??_C@_0BM@LIKDCEKJ@get?5IP_MULTICAST_TTL?5failed@ 1000f3ac     TwoStacksPlainDatagramSocketImpl.obj
 0002:000013c8       ??_C@_0BB@FCPOINAD@not?5in?5multicast@ 1000f3c8     TwoStacksPlainDatagramSocketImpl.obj
 0002:000013dc       ??_C@_0DA@OBEPBCCJ@Can?8t?5join?5an?5IPv4?5group?5on?5an?5@ 1000f3dc     TwoStacksPlainDatagramSocketImpl.obj
 0002:0000140c       ??_C@_0BL@KIMGBHOL@get?5IP_MULTICAST_IF?5failed@ 1000f40c     TwoStacksPlainDatagramSocketImpl.obj
 0002:00001428       ??_C@_0CK@FKKDPICG@no?5Inet4Address?5associated?5with@ 1000f428     TwoStacksPlainDatagramSocketImpl.obj
 0002:00001454       ??_C@_0DE@NGNCLOOP@IP_ADD_MEMBERSHIP?5failed?5?$CIout?5o@ 1000f454     TwoStacksPlainDatagramSocketImpl.obj
 0002:00001488       ??_C@_0BG@JBKBCMEL@error?5setting?5options@ 1000f488     TwoStacksPlainDatagramSocketImpl.obj
 0002:000014a0       ??_C@_0BC@JFLIBEAA@not?5in6?5multicast@ 1000f4a0     TwoStacksPlainDatagramSocketImpl.obj
 0002:000014b4       ??_C@_0BD@DCFJIHFI@IPv6?5not?5supported@ 1000f4b4     TwoStacksPlainDatagramSocketImpl.obj
 0002:000014c8       ??_C@_0CK@FBGIOLD@Can?8t?5join?5an?5IPv6?5group?5on?5a?5I@ 1000f4c8     TwoStacksPlainDatagramSocketImpl.obj
 0002:000014f4       ??_C@_0BN@CJPJHKGI@get?5IPV6_MULTICAST_IF?5failed@ 1000f4f4     TwoStacksPlainDatagramSocketImpl.obj
 0002:00001514       ??_C@_0BD@OLPOJDPI@get?5ifindex?5failed@ 1000f514     TwoStacksPlainDatagramSocketImpl.obj
 0002:00001528       ??_C@_03FCLDNGNL@TCP@      1000f528     TwoStacksPlainSocketImpl.obj
 0002:0000152c       ??_C@_09NOFGBFHM@localport@ 1000f52c     TwoStacksPlainSocketImpl.obj
 0002:00001538       ??_C@_0BI@PLIDPFNP@Ljava?1net?1ServerSocket?$DL@ 1000f538     TwoStacksPlainSocketImpl.obj
 0002:00001550       ??_C@_0N@DOLJHIMH@serverSocket@ 1000f550     TwoStacksPlainSocketImpl.obj
 0002:00001560       ??_C@_0P@BEFKEEJP@null?5fd?5object@ 1000f560     TwoStacksPlainSocketImpl.obj
 0002:00001570       ??_C@_0BA@FDCHHAEF@null?5fd1?5object@ 1000f570     TwoStacksPlainSocketImpl.obj
 0002:00001580       ??_C@_0BP@FPBJDHAC@inet?5address?5argument?5is?5null?4@ 1000f580     TwoStacksPlainSocketImpl.obj
 0002:000015a0       ??_C@_0BI@CCNHNILJ@Destination?5unreachable@ 1000f5a0     TwoStacksPlainSocketImpl.obj
 0002:000015b8       ??_C@_0BG@KFNCOJOM@inet?5address?5argument@ 1000f5b8     TwoStacksPlainSocketImpl.obj
 0002:000015d0       ??_C@_0CA@KIKJKBOB@getsockname?5in?5plain?5socketBind@ 1000f5d0     TwoStacksPlainSocketImpl.obj
 0002:000015f0       ??_C@_0P@HOPPFJIC@socket?5address@ 1000f5f0     TwoStacksPlainSocketImpl.obj
 0002:00001600       ??_C@_0P@LEIDGPMC@socket?5is?5null@ 1000f600     TwoStacksPlainSocketImpl.obj
 0002:00001610       ??_C@_0BJ@CKIILKAP@socket?5address?5or?5fd?5obj@ 1000f610     TwoStacksPlainSocketImpl.obj
 0002:0000162c       ??_C@_0O@EIDFHCCL@select?5failed@ 1000f62c     TwoStacksPlainSocketImpl.obj
 0002:0000163c       ??_C@_0BG@NLEJABIB@socket?5already?5closed@ 1000f63c     TwoStacksPlainSocketImpl.obj
 0002:00001654       ??_C@_0BH@OLFAGGPP@setsockopt?5SO_RCVTIMEO@ 1000f654     TwoStacksPlainSocketImpl.obj
 0002:0000166c       ??_C@_0DB@PPHBIKEI@Option?5not?5supported?5by?5TwoStac@ 1000f66c     TwoStacksPlainSocketImpl.obj
 0002:000016a0       ??_C@_0CC@HBHBHFNC@failed?5to?5initialize?5net?5librar@ 1000f6a0     net_util.obj
 0002:000016c4       ??_C@_0BP@JABHMODJ@java?1lang?1UnsatisfiedLinkError@ 1000f6c4     net_util.obj
 0002:000016e4       ??_C@_0BG@CGIGLAGP@?$CILjava?1lang?1String?$DL?$CJZ@ 1000f6e4     net_util.obj
 0002:000016fc       ??_C@_0L@HKKDKOBF@getBoolean@ 1000f6fc     net_util.obj
 0002:00001708       ??_C@_0BJ@OCGKBLBN@java?4net?4preferIPv4Stack@ 1000f708     net_util.obj
 0002:00001724       ??_C@_0BL@KNKNLGPI@InetAddress?5holder?5is?5null@ 1000f724     net_util.obj
 0002:0000195c       ??_C@_0BC@HFNFNKAI@Permission?5denied@ 1000f95c     net_util_md.obj
 0002:00001970       ??_C@_0O@GLDCGPDO@BindException@ 1000f970     net_util_md.obj
 0002:00001980       ??_C@_0BH@LOKACPE@Address?5already?5in?5use@ 1000f980     net_util_md.obj
 0002:00001998       ??_C@_0CA@NBHADPNL@Cannot?5assign?5requested?5address@ 1000f998     net_util_md.obj
 0002:000019b8       ??_C@_0DA@KDGLCJJO@Address?5family?5not?5supported?5by@ 1000f9b8     net_util_md.obj
 0002:000019e8       ??_C@_0BO@BMABNIPB@Operation?5already?5in?5progress@ 1000f9e8     net_util_md.obj
 0002:00001a08       ??_C@_0CB@DJAOADN@Software?5caused?5connection?5abor@ 1000fa08     net_util_md.obj
 0002:00001a2c       ??_C@_0BB@CICOPLDE@ConnectException@ 1000fa2c     net_util_md.obj
 0002:00001a40       ??_C@_0BD@NPDMPPFP@Connection?5refused@ 1000fa40     net_util_md.obj
 0002:00001a54       ??_C@_0BJ@FJAMCHKE@Connection?5reset?5by?5peer@ 1000fa54     net_util_md.obj
 0002:00001a70       ??_C@_0BN@HFCIEIME@Destination?5address?5required@ 1000fa70     net_util_md.obj
 0002:00001a90       ??_C@_0M@LOEHLCJD@Bad?5address@ 1000fa90     net_util_md.obj
 0002:00001a9c       ??_C@_0N@OHOPOBEF@Host?5is?5down@ 1000fa9c     net_util_md.obj
 0002:00001aac       ??_C@_0BH@PBADJGIL@NoRouteToHostException@ 1000faac     net_util_md.obj
 0002:00001ac4       ??_C@_0BB@PFBILCPA@No?5route?5to?5host@ 1000fac4     net_util_md.obj
 0002:00001ad8       ??_C@_0BK@LBMNDGCG@Operation?5now?5in?5progress@ 1000fad8     net_util_md.obj
 0002:00001af4       ??_C@_0BK@FJBOAFDK@Interrupted?5function?5call@ 1000faf4     net_util_md.obj
 0002:00001b10       ??_C@_0BB@HMGGCEBG@Invalid?5argument@ 1000fb10     net_util_md.obj
 0002:00001b24       ??_C@_0BM@CCONNCKE@Socket?5is?5already?5connected@ 1000fb24     net_util_md.obj
 0002:00001b40       ??_C@_0BE@INBJMKGG@Too?5many?5open?5files@ 1000fb40     net_util_md.obj
 0002:00001b58       ??_C@_0EN@MMGGBIMI@The?5message?5is?5larger?5than?5the?5@ 1000fb58     net_util_md.obj
 0002:00001ba8       ??_C@_0BA@LPIEBGEK@Network?5is?5down@ 1000fba8     net_util_md.obj
 0002:00001bb8       ??_C@_0CE@JHDCOCF@Network?5dropped?5connection?5on?5r@ 1000fbb8     net_util_md.obj
 0002:00001bdc       ??_C@_0BH@CIEOBPFM@Network?5is?5unreachable@ 1000fbdc     net_util_md.obj
 0002:00001bf4       ??_C@_0DJ@FJOKEEBP@No?5buffer?5space?5available?5?$CImaxi@ 1000fbf4     net_util_md.obj
 0002:00001c30       ??_C@_0BE@NEGCDJON@Bad?5protocol?5option@ 1000fc30     net_util_md.obj
 0002:00001c44       ??_C@_0BI@ILAOGBJJ@Socket?5is?5not?5connected@ 1000fc44     net_util_md.obj
 0002:00001c5c       ??_C@_0BO@PFGGHOGH@Socket?5operation?5on?5nonsocket@ 1000fc5c     net_util_md.obj
 0002:00001c7c       ??_C@_0BI@EDJAHLMH@Operation?5not?5supported@ 1000fc7c     net_util_md.obj
 0002:00001c94       ??_C@_0BD@LPHIGPM@Too?5many?5processes@ 1000fc94     net_util_md.obj
 0002:00001ca8       ??_C@_0BH@JNBKLLAJ@Protocol?5not?5supported@ 1000fca8     net_util_md.obj
 0002:00001cc0       ??_C@_0BP@PDKJLOAE@Protocol?5wrong?5type?5for?5socket@ 1000fcc0     net_util_md.obj
 0002:00001ce0       ??_C@_0CC@DAIJOIKC@Cannot?5send?5after?5socket?5shutdo@ 1000fce0     net_util_md.obj
 0002:00001d04       ??_C@_0BK@LMAIHBL@Socket?5type?5not?5supported@ 1000fd04     net_util_md.obj
 0002:00001d20       ??_C@_0BF@IBBHAGLD@Connection?5timed?5out@ 1000fd20     net_util_md.obj
 0002:00001d38       ??_C@_0BF@EHICFGGJ@Class?5type?5not?5found@ 1000fd38     net_util_md.obj
 0002:00001d50       ??_C@_0CB@EPFKGNAK@Resource?5temporarily?5unavailabl@ 1000fd50     net_util_md.obj
 0002:00001d74       ??_C@_0P@CAFMJNJH@Host?5not?5found@ 1000fd74     net_util_md.obj
 0002:00001d84       ??_C@_0BO@GICNLCFB@Insufficient?5memory?5available@ 1000fd84     net_util_md.obj
 0002:00001da4       ??_C@_0CI@CFJNLLNI@Successful?5WSAStartup?5not?5yet?5p@ 1000fda4     net_util_md.obj
 0002:00001dcc       ??_C@_0CN@KFPNHBIN@Valid?5name?0?5no?5data?5record?5of?5r@ 1000fdcc     net_util_md.obj
 0002:00001dfc       ??_C@_0BP@BOOHLDLA@This?5is?5a?5nonrecoverable?5error@ 1000fdfc     net_util_md.obj
 0002:00001e1c       ??_C@_0CB@PLJNFILF@Network?5subsystem?5is?5unavailabl@ 1000fe1c     net_util_md.obj
 0002:00001e40       ??_C@_0CA@DOKOCCFB@Nonauthoritative?5host?5not?5found@ 1000fe40     net_util_md.obj
 0002:00001e60       ??_C@_0CB@GHMLGJBG@Winsock?4dll?5version?5out?5of?5rang@ 1000fe60     net_util_md.obj
 0002:00001e84       ??_C@_0BO@ILFFGILJ@Graceful?5shutdown?5in?5progress@ 1000fe84     net_util_md.obj
 0002:00001ea4       ??_C@_0BN@KGMIDOOK@Overlapped?5operation?5aborted@ 1000fea4     net_util_md.obj
 0002:00001ec4       ??_C@_0BH@GDIHDDN@no?5further?5information@ 1000fec4     net_util_md.obj
 0002:00001edc       ??_C@_06DJHOIPC@?$CFs?3?5?$CFs@ 1000fedc     net_util_md.obj
 0002:00001ee4       ??_C@_0CL@EIMGMHJP@Unrecognized?5Windows?5Sockets?5er@ 1000fee4     net_util_md.obj
 0002:00001f10       ??_C@_0BA@EOEGOLGE@SocketException@ 1000ff10     net_util_md.obj
 0002:00001f20       ??_C@_09ELLCMIIO@java?1net?1@ 1000ff20     net_util_md.obj
 0002:00001f2c       ??_C@_04HDOCAJNK@?$CFs?$CFs@ 1000ff2c     net_util_md.obj
 0002:00001f34       ??_C@_0DB@GKAPFAKD@SYSTEM?2CurrentControlSet?2Servic@ 1000ff34     net_util_md.obj
 0002:00001f68       ??_C@_0DH@IMHEAAEF@SYSTEM?2CurrentControlSet?2Servic@ 1000ff68     net_util_md.obj
 0002:00001fa0       ??_C@_0L@JFBEJJHM@DefaultTOS@ 1000ffa0     net_util_md.obj
 0002:00001fac       ??_C@_0BM@PJBFLPGI@Protocol?5family?5unavailable@ 1000ffac     net_util_md.obj
 0002:00001fc8       ??_C@_0M@JMCMHGIK@MaxUserPort@ 1000ffc8     portconfig.obj
 0002:00001fd4       _in6addr_any               1000ffd4     ws2_32:indef.obj
 0002:00001ff0       __sz_Secur32_dll           1000fff0     secur32:Secur32.dll
 0002:00002000       __sz_IPHLPAPI_DLL          10010000     iphlpapi:IPHLPAPI.DLL
 0002:00002010       ??_C@_1BK@DBDEIDLH@?$AAK?$AAE?$AAR?$AAN?$AAE?$AAL?$AA3?$AA2?$AA?4?$AAD?$AAL?$AAL@ 10010010     delayimp:delayhlp.obj
 0002:0000202c       ??_C@_0BI@OMNLIJDB@AcquireSRWLockExclusive@ 1001002c     delayimp:delayhlp.obj
 0002:00002044       ??_C@_0BI@HMIEPCNJ@ReleaseSRWLockExclusive@ 10010044     delayimp:delayhlp.obj
 0002:0000205c       ___pfnDliNotifyHook2       1001005c     delayimp:delayhk2.obj
 0002:00002060       ___pfnDliFailureHook2      10010060     delayimp:delayhk1.obj
 0002:00002064       __pDefaultRawDllMain       10010064     MSVCRT:dll_dllmain.obj
 0002:00002064       __pRawDllMain              10010064     MSVCRT:dll_dllmain.obj
 0002:00002068       __load_config_used         10010068     MSVCRT:loadcfg.obj
 0002:000021c0       ___safe_se_handler_table   100101c0     <linker-defined>
 0002:000021c4       ___volatile_metadata       100101c4     <linker-defined>
 0002:00002598       ___rtc_iaa                 10010598     MSVCRT:initsect.obj
 0002:0000259c       ___rtc_izz                 1001059c     MSVCRT:initsect.obj
 0002:000025a0       ___rtc_taa                 100105a0     MSVCRT:initsect.obj
 0002:000025a4       ___rtc_tzz                 100105a4     MSVCRT:initsect.obj
 0002:0000262c       __DELAY_IMPORT_DESCRIPTOR_secur32_dll 1001062c     secur32:Secur32.dll
 0002:0000264c       __DELAY_IMPORT_DESCRIPTOR_iphlpapi_dll 1001064c     iphlpapi:IPHLPAPI.DLL
 0002:0000266c       __NULL_DELAY_IMPORT_DESCRIPTOR 1001066c     secur32:Secur32.dll
 0002:000026bc       \177IPHLPAPI_NULL_THUNK_DATA_DLN 100106bc     iphlpapi:IPHLPAPI.DLL
 0002:000026d4       \177Secur32_NULL_THUNK_DATA_DLN 100106d4     secur32:Secur32.dll
 0002:00002838       \177Secur32_NULL_THUNK_DATA_DLB 10010838     secur32:Secur32.dll
 0002:00002850       \177IPHLPAPI_NULL_THUNK_DATA_DLB 10010850     iphlpapi:IPHLPAPI.DLL
 0002:00004a60       __IMPORT_DESCRIPTOR_WS2_32 10012a60     ws2_32:WS2_32.dll
 0002:00004a74       __IMPORT_DESCRIPTOR_jvm    10012a74     jvm:jvm.dll
 0002:00004a88       __IMPORT_DESCRIPTOR_java   10012a88     java:java.dll
 0002:00004a9c       __IMPORT_DESCRIPTOR_ADVAPI32 10012a9c     advapi32:ADVAPI32.dll
 0002:00004ab0       __IMPORT_DESCRIPTOR_KERNEL32 10012ab0     kernel32:KERNEL32.dll
 0002:00004ac4       __IMPORT_DESCRIPTOR_VCRUNTIME140 10012ac4     vcruntime:VCRUNTIME140.dll
 0002:00004ad8       __IMPORT_DESCRIPTOR_api-ms-win-crt-string-l1-1-0 10012ad8     ucrt:api-ms-win-crt-string-l1-1-0.dll
 0002:00004aec       __IMPORT_DESCRIPTOR_api-ms-win-crt-stdio-l1-1-0 10012aec     ucrt:api-ms-win-crt-stdio-l1-1-0.dll
 0002:00004b00       __IMPORT_DESCRIPTOR_api-ms-win-crt-heap-l1-1-0 10012b00     ucrt:api-ms-win-crt-heap-l1-1-0.dll
 0002:00004b14       __IMPORT_DESCRIPTOR_api-ms-win-crt-runtime-l1-1-0 10012b14     ucrt:api-ms-win-crt-runtime-l1-1-0.dll
 0002:00004b28       __NULL_IMPORT_DESCRIPTOR   10012b28     ws2_32:WS2_32.dll
 0003:00000008       _isRcvTimeoutSupported     10014008     net_util_md.obj
 0003:00000094       ___security_cookie_complement 10014094     MSVCRT:gs_cookie.obj
 0003:00000098       ___security_cookie         10014098     MSVCRT:gs_cookie.obj
 0003:0000009c       ___scrt_native_dllmain_reason 1001409c     MSVCRT:utility.obj
 0003:000000a0       ___isa_enabled             100140a0     MSVCRT:cpu_disp.obj
 0003:000000a4       ___scrt_ucrt_dll_is_in_use 100140a4     MSVCRT:ucrt_stubs.obj
 0003:000000a8       __imp__IcmpSendEcho@32     100140a8     iphlpapi:IPHLPAPI.DLL
 0003:000000ac       __imp__NotifyAddrChange@8  100140ac     iphlpapi:IPHLPAPI.DLL
 0003:000000b0       __imp__GetAdaptersAddresses@20 100140b0     iphlpapi:IPHLPAPI.DLL
 0003:000000b4       __imp__GetFriendlyIfIndex@4 100140b4     iphlpapi:IPHLPAPI.DLL
 0003:000000b8       __imp__GetIpAddrTable@12   100140b8     iphlpapi:IPHLPAPI.DLL
 0003:000000bc       __imp__GetIfTable@12       100140bc     iphlpapi:IPHLPAPI.DLL
 0003:000000c0       __imp__IcmpCreateFile@0    100140c0     iphlpapi:IPHLPAPI.DLL
 0003:000000c4       __imp__Icmp6SendEcho2@48   100140c4     iphlpapi:IPHLPAPI.DLL
 0003:000000c8       __imp__IcmpCloseHandle@4   100140c8     iphlpapi:IPHLPAPI.DLL
 0003:000000cc       __imp__GetAdaptersInfo@8   100140cc     iphlpapi:IPHLPAPI.DLL
 0003:000000d0       __imp__IcmpSendEcho2Ex@48  100140d0     iphlpapi:IPHLPAPI.DLL
 0003:000000d4       __imp__Icmp6CreateFile@0   100140d4     iphlpapi:IPHLPAPI.DLL
 0003:000000d8       \177IPHLPAPI_NULL_THUNK_DATA_DLA 100140d8     iphlpapi:IPHLPAPI.DLL
 0003:000000dc       __imp__CompleteAuthToken@8 100140dc     secur32:Secur32.dll
 0003:000000e0       __imp__InitializeSecurityContextA@48 100140e0     secur32:Secur32.dll
 0003:000000e4       __imp__FreeCredentialsHandle@4 100140e4     secur32:Secur32.dll
 0003:000000e8       __imp__AcquireCredentialsHandleA@36 100140e8     secur32:Secur32.dll
 0003:000000ec       __imp__DeleteSecurityContext@4 100140ec     secur32:Secur32.dll
 0003:000000f0       \177Secur32_NULL_THUNK_DATA_DLA 100140f0     secur32:Secur32.dll
 0003:000001f8       __hmod__Secur32_dll        100141f8     secur32:Secur32.dll
 0003:000001fc       __hmod__IPHLPAPI_DLL       100141fc     iphlpapi:IPHLPAPI.DLL
 0003:00000200       ?DloadKernel32@@3PAUHINSTANCE__@@A 10014200     delayimp:delayhlp.obj
 0003:00000204       ?DloadAcquireSRWLockExclusive@@3P6GXPAK@ZA 10014204     delayimp:delayhlp.obj
 0003:00000208       ?DloadReleaseSRWLockExclusive@@3P6GXPAK@ZA 10014208     delayimp:delayhlp.obj
 0003:0000020c       ?DloadSrwLock@@3KA         1001420c     delayimp:delayhlp.obj
 0003:00000210       ?DloadSectionLockCount@@3KA 10014210     delayimp:delayhlp.obj
 0003:00000214       ?DloadSectionOldProtection@@3KA 10014214     delayimp:delayhlp.obj
 0003:00000218       ?DloadSectionCommitPermanent@@3KA 10014218     delayimp:delayhlp.obj
 0003:00000540       ?__type_info_root_node@@3U__type_info_node@@A 10014540     MSVCRT:tncleanup.obj
 0003:00000548       ___scrt_current_native_startup_state 10014548     MSVCRT:utility.obj
 0003:0000054c       ___scrt_native_startup_lock 1001454c     MSVCRT:utility.obj
 0003:0000056c       ___scrt_debugger_hook_flag 1001456c     MSVCRT:utility_desktop.obj
 0003:00000570       ___isa_available           10014570     MSVCRT:cpu_disp.obj
 0003:00000574       ___favor                   10014574     MSVCRT:cpu_disp.obj
 0003:00000578       _psi_lastfdID              10014578     <common>
 0003:0000057c       _psi_serverSocketID        1001457c     <common>
 0003:00000580       _psi_trafficClassID        10014580     <common>
 0003:00000584       _psi_fd1ID                 10014584     <common>
 0003:00000588       _psi_localportID           10014588     <common>
 0003:0000058c       _psi_portID                1001458c     <common>
 0003:00000590       _psi_addressID             10014590     <common>
 0003:00000594       _psi_fdID                  10014594     <common>
 0003:00000598       _psi_timeoutID             10014598     <common>
 0003:0000059c       _pdsi_connected            1001459c     <common>
 0003:000005a0       _pdsi_localPortID          100145a0     <common>
 0003:000005a4       _pdsi_timeoutID            100145a4     <common>
 0003:000005a8       _pdsi_lastfdID             100145a8     <common>
 0003:000005ac       _pdsi_fduseID              100145ac     <common>
 0003:000005b0       _pdsi_fd1ID                100145b0     <common>
 0003:000005b4       _pdsi_fdID                 100145b4     <common>
 0003:000005b8       _ni_ibmaskID               100145b8     <common>
 0003:000005bc       _ni_ibbroadcastID          100145bc     <common>
 0003:000005c0       _ni_ibaddressID            100145c0     <common>
 0003:000005c4       _ni_ibctrID                100145c4     <common>
 0003:000005c8       _ni_ibcls                  100145c8     <common>
 0003:000005cc       _ni_childsID               100145cc     <common>
 0003:000005d0       _ni_displayNameID          100145d0     <common>
 0003:000005d4       _ni_bindsID                100145d4     <common>
 0003:000005d8       _ni_ctor                   100145d8     <common>
 0003:000005dc       _ni_addrsID                100145dc     <common>
 0003:000005e0       _ni_indexID                100145e0     <common>
 0003:000005e4       _ni_nameID                 100145e4     <common>
 0003:000005e8       _ni_class                  100145e8     <common>
 0003:000005ec       _ia_holderID               100145ec     <common>
 0003:000005f0       _iac_class                 100145f0     <common>
 0003:000005f4       _ia_preferIPv6AddressID    100145f4     <common>
 0003:000005f8       _iac_origHostNameID        100145f8     <common>
 0003:000005fc       _iac_hostNameID            100145fc     <common>
 0003:00000600       _iac_familyID              10014600     <common>
 0003:00000604       _iac_addressID             10014604     <common>
 0003:00000608       _ia_class                  10014608     <common>
 0003:0000060c       _ia6_ctrID                 1001460c     <common>
 0003:00000610       _ia6_scopeifnameID         10014610     <common>
 0003:00000614       _ia6_scopeidsetID          10014614     <common>
 0003:00000618       _ia6_cachedscopeidID       10014618     <common>
 0003:0000061c       _ia6_scopeidID             1001461c     <common>
 0003:00000620       _ia6_ipaddressID           10014620     <common>
 0003:00000624       _ia6_holder6ID             10014624     <common>
 0003:00000628       _ia6_class                 10014628     <common>
 0003:0000062c       _ia4_ctrID                 1001462c     <common>
 0003:00000630       _ia4_class                 10014630     <common>
 0003:00000638       ?_OptionsStorage@?1??__local_stdio_scanf_options@@9@9 10014638     <common>
 0003:00000640       ?_OptionsStorage@?1??__local_stdio_printf_options@@9@9 10014640     <common>
 0003:00000648       _dp_bufLengthID            10014648     <common>
 0003:0000064c       _dp_lengthID               1001464c     <common>
 0003:00000650       _dp_offsetID               10014650     <common>
 0003:00000654       _dp_bufID                  10014654     <common>
 0003:00000658       _dp_portID                 10014658     <common>
 0003:0000065c       _dp_addressID              1001465c     <common>
 0003:00000660       ___dyn_tls_init_callback   10014660     <common>

 entry point at        0001:0000bf90

 Static symbols

 0000:fffe9000       .debug$S                   10000000     net.exp
 0000:fffe9000       .debug$S                   10000000     vcruntime:VCRUNTIME140.dll
 0000:fffe9000       .debug$S                   10000000     vcruntime:VCRUNTIME140.dll
 0000:fffe9000       .debug$S                   10000000     vcruntime:VCRUNTIME140.dll
 0000:fffe9000       .debug$S                   10000000     vcruntime:VCRUNTIME140.dll
 0000:fffe9000       .debug$S                   10000000     vcruntime:VCRUNTIME140.dll
 0000:fffe9000       .debug$S                   10000000     vcruntime:VCRUNTIME140.dll
 0000:fffe9000       .debug$S                   10000000     vcruntime:VCRUNTIME140.dll
 0000:fffe9000       .debug$S                   10000000     vcruntime:VCRUNTIME140.dll
 0000:fffe9000       .debug$S                   10000000     ucrt:api-ms-win-crt-heap-l1-1-0.dll
 0000:fffe9000       .debug$S                   10000000     ucrt:api-ms-win-crt-heap-l1-1-0.dll
 0000:fffe9000       .debug$S                   10000000     ucrt:api-ms-win-crt-heap-l1-1-0.dll
 0000:fffe9000       .debug$S                   10000000     ucrt:api-ms-win-crt-heap-l1-1-0.dll
 0000:fffe9000       .debug$S                   10000000     ucrt:api-ms-win-crt-runtime-l1-1-0.dll
 0000:fffe9000       .debug$S                   10000000     ucrt:api-ms-win-crt-runtime-l1-1-0.dll
 0000:fffe9000       .debug$S                   10000000     ucrt:api-ms-win-crt-runtime-l1-1-0.dll
 0000:fffe9000       .debug$S                   10000000     ucrt:api-ms-win-crt-runtime-l1-1-0.dll
 0000:fffe9000       .debug$S                   10000000     ucrt:api-ms-win-crt-runtime-l1-1-0.dll
 0000:fffe9000       .debug$S                   10000000     ucrt:api-ms-win-crt-runtime-l1-1-0.dll
 0000:fffe9000       .debug$S                   10000000     ucrt:api-ms-win-crt-runtime-l1-1-0.dll
 0000:fffe9000       .debug$S                   10000000     ucrt:api-ms-win-crt-runtime-l1-1-0.dll
 0000:fffe9000       .debug$S                   10000000     ucrt:api-ms-win-crt-runtime-l1-1-0.dll
 0000:fffe9000       .debug$S                   10000000     ucrt:api-ms-win-crt-runtime-l1-1-0.dll
 0000:fffe9000       .debug$S                   10000000     ucrt:api-ms-win-crt-runtime-l1-1-0.dll
 0000:fffe9000       .debug$S                   10000000     ucrt:api-ms-win-crt-runtime-l1-1-0.dll
 0000:fffe9000       .debug$S                   10000000     ucrt:api-ms-win-crt-runtime-l1-1-0.dll
 0000:fffe9000       .debug$S                   10000000     ucrt:api-ms-win-crt-stdio-l1-1-0.dll
 0000:fffe9000       .debug$S                   10000000     ucrt:api-ms-win-crt-stdio-l1-1-0.dll
 0000:fffe9000       .debug$S                   10000000     ucrt:api-ms-win-crt-stdio-l1-1-0.dll
 0000:fffe9000       .debug$S                   10000000     ucrt:api-ms-win-crt-stdio-l1-1-0.dll
 0000:fffe9000       .debug$S                   10000000     ucrt:api-ms-win-crt-stdio-l1-1-0.dll
 0000:fffe9000       .debug$S                   10000000     ucrt:api-ms-win-crt-string-l1-1-0.dll
 0000:fffe9000       .debug$S                   10000000     ucrt:api-ms-win-crt-string-l1-1-0.dll
 0000:fffe9000       .debug$S                   10000000     ucrt:api-ms-win-crt-string-l1-1-0.dll
 0000:fffe9000       .debug$S                   10000000     ucrt:api-ms-win-crt-string-l1-1-0.dll
 0000:fffe9000       .debug$S                   10000000     ucrt:api-ms-win-crt-string-l1-1-0.dll
 0000:fffe9000       .debug$S                   10000000     ucrt:api-ms-win-crt-string-l1-1-0.dll
 0000:fffe9000       .debug$S                   10000000     ucrt:api-ms-win-crt-string-l1-1-0.dll
 0000:fffe9000       .debug$S                   10000000     ucrt:api-ms-win-crt-string-l1-1-0.dll
 0000:fffe9000       .debug$S                   10000000     ucrt:api-ms-win-crt-string-l1-1-0.dll
 0000:fffe9000       .debug$S                   10000000     ucrt:api-ms-win-crt-string-l1-1-0.dll
 0000:fffe9000       .debug$S                   10000000     ucrt:api-ms-win-crt-string-l1-1-0.dll
 0000:fffe9000       .debug$S                   10000000     advapi32:ADVAPI32.dll
 0000:fffe9000       .debug$S                   10000000     advapi32:ADVAPI32.dll
 0000:fffe9000       .debug$S                   10000000     advapi32:ADVAPI32.dll
 0000:fffe9000       .debug$S                   10000000     iphlpapi:IPHLPAPI.DLL
 0000:fffe9000       .debug$S                   10000000     iphlpapi:IPHLPAPI.DLL
 0000:fffe9000       .debug$S                   10000000     iphlpapi:IPHLPAPI.DLL
 0000:fffe9000       .debug$S                   10000000     iphlpapi:IPHLPAPI.DLL
 0000:fffe9000       .debug$S                   10000000     iphlpapi:IPHLPAPI.DLL
 0000:fffe9000       .debug$S                   10000000     iphlpapi:IPHLPAPI.DLL
 0000:fffe9000       .debug$S                   10000000     iphlpapi:IPHLPAPI.DLL
 0000:fffe9000       .debug$S                   10000000     iphlpapi:IPHLPAPI.DLL
 0000:fffe9000       .debug$S                   10000000     iphlpapi:IPHLPAPI.DLL
 0000:fffe9000       .debug$S                   10000000     iphlpapi:IPHLPAPI.DLL
 0000:fffe9000       .debug$S                   10000000     iphlpapi:IPHLPAPI.DLL
 0000:fffe9000       .debug$S                   10000000     iphlpapi:IPHLPAPI.DLL
 0000:fffe9000       .debug$S                   10000000     kernel32:KERNEL32.dll
 0000:fffe9000       .debug$S                   10000000     kernel32:KERNEL32.dll
 0000:fffe9000       .debug$S                   10000000     kernel32:KERNEL32.dll
 0000:fffe9000       .debug$S                   10000000     kernel32:KERNEL32.dll
 0000:fffe9000       .debug$S                   10000000     kernel32:KERNEL32.dll
 0000:fffe9000       .debug$S                   10000000     kernel32:KERNEL32.dll
 0000:fffe9000       .debug$S                   10000000     kernel32:KERNEL32.dll
 0000:fffe9000       .debug$S                   10000000     kernel32:KERNEL32.dll
 0000:fffe9000       .debug$S                   10000000     kernel32:KERNEL32.dll
 0000:fffe9000       .debug$S                   10000000     kernel32:KERNEL32.dll
 0000:fffe9000       .debug$S                   10000000     kernel32:KERNEL32.dll
 0000:fffe9000       .debug$S                   10000000     kernel32:KERNEL32.dll
 0000:fffe9000       .debug$S                   10000000     kernel32:KERNEL32.dll
 0000:fffe9000       .debug$S                   10000000     kernel32:KERNEL32.dll
 0000:fffe9000       .debug$S                   10000000     kernel32:KERNEL32.dll
 0000:fffe9000       .debug$S                   10000000     kernel32:KERNEL32.dll
 0000:fffe9000       .debug$S                   10000000     kernel32:KERNEL32.dll
 0000:fffe9000       .debug$S                   10000000     kernel32:KERNEL32.dll
 0000:fffe9000       .debug$S                   10000000     kernel32:KERNEL32.dll
 0000:fffe9000       .debug$S                   10000000     kernel32:KERNEL32.dll
 0000:fffe9000       .debug$S                   10000000     kernel32:KERNEL32.dll
 0000:fffe9000       .debug$S                   10000000     kernel32:KERNEL32.dll
 0000:fffe9000       .debug$S                   10000000     kernel32:KERNEL32.dll
 0000:fffe9000       .debug$S                   10000000     kernel32:KERNEL32.dll
 0000:fffe9000       .debug$S                   10000000     kernel32:KERNEL32.dll
 0000:fffe9000       .debug$S                   10000000     kernel32:KERNEL32.dll
 0000:fffe9000       .debug$S                   10000000     kernel32:KERNEL32.dll
 0000:fffe9000       .debug$S                   10000000     kernel32:KERNEL32.dll
 0000:fffe9000       .debug$S                   10000000     kernel32:KERNEL32.dll
 0000:fffe9000       .debug$S                   10000000     kernel32:KERNEL32.dll
 0000:fffe9000       .debug$S                   10000000     kernel32:KERNEL32.dll
 0000:fffe9000       .debug$S                   10000000     kernel32:KERNEL32.dll
 0000:fffe9000       .debug$S                   10000000     kernel32:KERNEL32.dll
 0000:fffe9000       .debug$S                   10000000     secur32:Secur32.dll
 0000:fffe9000       .debug$S                   10000000     secur32:Secur32.dll
 0000:fffe9000       .debug$S                   10000000     secur32:Secur32.dll
 0000:fffe9000       .debug$S                   10000000     secur32:Secur32.dll
 0000:fffe9000       .debug$S                   10000000     secur32:Secur32.dll
 0000:fffe9000       .debug$S                   10000000     ws2_32:WS2_32.dll
 0000:fffe9000       .debug$S                   10000000     ws2_32:WS2_32.dll
 0000:fffe9000       .debug$S                   10000000     ws2_32:WS2_32.dll
 0000:fffe9000       .debug$S                   10000000     ws2_32:WS2_32.dll
 0000:fffe9000       .debug$S                   10000000     ws2_32:WS2_32.dll
 0000:fffe9000       .debug$S                   10000000     ws2_32:WS2_32.dll
 0000:fffe9000       .debug$S                   10000000     ws2_32:WS2_32.dll
 0000:fffe9000       .debug$S                   10000000     ws2_32:WS2_32.dll
 0000:fffe9000       .debug$S                   10000000     ws2_32:WS2_32.dll
 0000:fffe9000       .debug$S                   10000000     ws2_32:WS2_32.dll
 0000:fffe9000       .debug$S                   10000000     ws2_32:WS2_32.dll
 0000:fffe9000       .debug$S                   10000000     ws2_32:WS2_32.dll
 0000:fffe9000       .debug$S                   10000000     ws2_32:WS2_32.dll
 0000:fffe9000       .debug$S                   10000000     ws2_32:WS2_32.dll
 0000:fffe9000       .debug$S                   10000000     ws2_32:WS2_32.dll
 0000:fffe9000       .debug$S                   10000000     ws2_32:WS2_32.dll
 0000:fffe9000       .debug$S                   10000000     ws2_32:WS2_32.dll
 0000:fffe9000       .debug$S                   10000000     ws2_32:WS2_32.dll
 0000:fffe9000       .debug$S                   10000000     ws2_32:WS2_32.dll
 0000:fffe9000       .debug$S                   10000000     ws2_32:WS2_32.dll
 0000:fffe9000       .debug$S                   10000000     ws2_32:WS2_32.dll
 0000:fffe9000       .debug$S                   10000000     ws2_32:WS2_32.dll
 0000:fffe9000       .debug$S                   10000000     ws2_32:WS2_32.dll
 0000:fffe9000       .debug$S                   10000000     ws2_32:WS2_32.dll
 0000:fffe9000       .debug$S                   10000000     ws2_32:WS2_32.dll
 0000:fffe9000       .debug$S                   10000000     ws2_32:WS2_32.dll
 0000:fffe9000       .debug$S                   10000000     ws2_32:WS2_32.dll
 0000:fffe9000       .debug$S                   10000000     ws2_32:WS2_32.dll
 0000:fffe9000       .debug$S                   10000000     ws2_32:WS2_32.dll
 0000:fffe9000       .debug$S                   10000000     ws2_32:WS2_32.dll
 0000:fffe9000       .debug$S                   10000000     ws2_32:WS2_32.dll
 0000:fffe9000       .debug$S                   10000000     ws2_32:WS2_32.dll
 0000:fffe9000       .debug$S                   10000000     ws2_32:WS2_32.dll
 0000:fffe9000       .debug$S                   10000000     ws2_32:WS2_32.dll
 0000:fffe9000       .debug$S                   10000000     ws2_32:WS2_32.dll
 0000:fffe9000       .debug$S                   10000000     ws2_32:WS2_32.dll
 0000:fffe9000       .debug$S                   10000000     ws2_32:WS2_32.dll
 0000:fffe9000       .debug$S                   10000000     jvm:jvm.dll
 0000:fffe9000       .debug$S                   10000000     jvm:jvm.dll
 0000:fffe9000       .debug$S                   10000000     jvm:jvm.dll
 0000:fffe9000       .debug$S                   10000000     java:java.dll
 0000:fffe9000       .debug$S                   10000000     java:java.dll
 0000:fffe9000       .debug$S                   10000000     java:java.dll
 0000:fffe9000       .debug$S                   10000000     java:java.dll
 0000:fffe9000       .debug$S                   10000000     java:java.dll
 0000:fffe9000       .debug$S                   10000000     java:java.dll
 0000:fffe9000       .debug$S                   10000000     java:java.dll
 0000:fffe9000       .debug$S                   10000000     java:java.dll
 0000:fffe9000       .debug$S                   10000000     java:java.dll
 0000:fffe9000       .debug$S                   10000000     java:java.dll
 0001:00000fa0       _purgeOutstandingICMP      10001fa0 f   DualStackPlainDatagramSocketImpl.obj
 0001:00001ccf       _WindowsVersionCheck       10002ccf f   Inet4AddressImpl.obj
 0001:00001df1       _ping4                     10002df1 f   Inet4AddressImpl.obj
 0001:00001f7d       _tcp_ping4                 10002f7d f   Inet4AddressImpl.obj
 0001:000029b9       _ping6                     100039b9 f   Inet6AddressImpl.obj
 0001:00002a8a       _tcp_ping6                 10003a8a f   Inet6AddressImpl.obj
 0001:000031da       _endSequence               100041da f   NTLMAuthSequence.obj
 0001:0000488b       _createNetworkInterfaceXP  1000588b f   NetworkInterface_winXP.obj
 0001:00004d19       _getAdapters               10005d19 f   NetworkInterface_winXP.obj
 0001:00004dea       _getAddrsFromAdapter       10005dea f   NetworkInterface_winXP.obj
 0001:00005318       _loadConfig                10006318 f   ResolverConfigurationImpl.obj
 0001:00007951       _checkLastFD               10008951 f   TwoStacksPlainDatagramSocketImpl.obj
 0001:00007c7b       _getFD                     10008c7b f   TwoStacksPlainDatagramSocketImpl.obj
 0001:00007cb0       _getFD1                    10008cb0 f   TwoStacksPlainDatagramSocketImpl.obj
 0001:00007ce5       _getIPv4NetworkInterface   10008ce5 f   TwoStacksPlainDatagramSocketImpl.obj
 0001:00007eef       _getIndexFromIf            10008eef f   TwoStacksPlainDatagramSocketImpl.obj
 0001:00007f44       _getInet4AddrFromIf        10008f44 f   TwoStacksPlainDatagramSocketImpl.obj
 0001:00007f94       _getInetAddrFromIf         10008f94 f   TwoStacksPlainDatagramSocketImpl.obj
 0001:0000833f       _isAdapterIpv6Enabled      1000933f f   TwoStacksPlainDatagramSocketImpl.obj
 0001:0000838d       _mcast_join_leave          1000938d f   TwoStacksPlainDatagramSocketImpl.obj
 0001:0000863d       _purgeOutstandingICMP      1000963d f   TwoStacksPlainDatagramSocketImpl.obj
 0001:00008712       _setMulticastInterface     10009712 f   TwoStacksPlainDatagramSocketImpl.obj
 0001:000088c6       _supportPortUnreachable    100098c6 f   TwoStacksPlainDatagramSocketImpl.obj
 0001:00009f73       _getFD                     1000af73 f   TwoStacksPlainSocketImpl.obj
 0001:00009fa8       _getFD1                    1000afa8 f   TwoStacksPlainSocketImpl.obj
 0001:0000b548       _getPortRange              1000c548 f   portconfig.obj
 0001:0000bc50       ?dllmain_crt_dispatch@@YGHQAUHINSTANCE__@@KQAX@Z 1000cc50 f   MSVCRT:dll_dllmain.obj
 0001:0000bca3       ?dllmain_crt_process_attach@@YAHQAUHINSTANCE__@@QAX@Z 1000cca3 f   MSVCRT:dll_dllmain.obj
 0001:0000bdaa       ?dllmain_crt_process_detach@@YAH_N@Z 1000cdaa f   MSVCRT:dll_dllmain.obj
 0001:0000be5a       ?dllmain_dispatch@@YAHQAUHINSTANCE__@@KQAX@Z 1000ce5a f   MSVCRT:dll_dllmain.obj
 0001:0000bf65       ?dllmain_raw@@YGHQAUHINSTANCE__@@KQAX@Z 1000cf65 f   MSVCRT:dll_dllmain.obj
 0001:0000c0d5       ___get_entropy             1000d0d5 f   MSVCRT:gs_support.obj
 0001:0000c1a2       ?find_pe_section@@YAPAU_IMAGE_SECTION_HEADER@@QAEI@Z 1000d1a2 f   MSVCRT:utility.obj
 0001:0000c600       $$000000                   1000d600     MSVCRT:sehprolg4.obj
 0002:00001740       _winsock_errors            1000f740     net_util_md.obj
 0002:00002128       _GS_ExceptionPointers      10010128     MSVCRT:gs_report.obj
 0002:000025a8       __sehtable$?dllmain_crt_process_attach@@YAHQAUHINSTANCE__@@QAX@Z 100105a8     MSVCRT:dll_dllmain.obj
 0002:000025c8       __sehtable$?dllmain_crt_process_detach@@YAH_N@Z 100105c8     MSVCRT:dll_dllmain.obj
 0002:000025f0       __sehtable$?dllmain_dispatch@@YAHQAUHINSTANCE__@@KQAX@Z 100105f0     MSVCRT:dll_dllmain.obj
 0002:00002610       __sehtable$___scrt_is_nonwritable_in_current_image 10010610     MSVCRT:utility.obj
 0002:00002880       .edata                     10010880     net.exp
 0002:000028a8       rgpv                       100108a8     net.exp
 0002:00002ae0       rgszName                   10010ae0     net.exp
 0002:00002d18       rgwOrd                     10010d18     net.exp
 0002:00002e34       szName                     10010e34     net.exp
 0002:00002e3c       $N00001                    10010e3c     net.exp
 0002:00002e4a       $N00002                    10010e4a     net.exp
 0002:00002e6f       $N00003                    10010e6f     net.exp
 0002:00002eaf       $N00004                    10010eaf     net.exp
 0002:00002ee9       $N00005                    10010ee9     net.exp
 0002:00002f27       $N00006                    10010f27     net.exp
 0002:00002f66       $N00007                    10010f66     net.exp
 0002:00002fa7       $N00008                    10010fa7     net.exp
 0002:00002fe7       $N00009                    10010fe7     net.exp
 0002:0000302b       $N00010                    1001102b     net.exp
 0002:00003071       $N00011                    10011071     net.exp
 0002:000030b7       $N00012                    100110b7     net.exp
 0002:000030fa       $N00013                    100110fa     net.exp
 0002:00003145       $N00014                    10011145     net.exp
 0002:00003183       $N00015                    10011183     net.exp
 0002:000031c9       $N00016                    100111c9     net.exp
 0002:000031fc       $N00017                    100111fc     net.exp
 0002:00003232       $N00018                    10011232     net.exp
 0002:00003263       $N00019                    10011263     net.exp
 0002:00003295       $N00020                    10011295     net.exp
 0002:000032d2       $N00021                    100112d2     net.exp
 0002:00003306       $N00022                    10011306     net.exp
 0002:0000333e       $N00023                    1001133e     net.exp
 0002:00003370       $N00024                    10011370     net.exp
 0002:000033a3       $N00025                    100113a3     net.exp
 0002:000033db       $N00026                    100113db     net.exp
 0002:00003411       $N00027                    10011411     net.exp
 0002:00003444       $N00028                    10011444     net.exp
 0002:0000347c       $N00029                    1001147c     net.exp
 0002:000034b1       $N00030                    100114b1     net.exp
 0002:000034e4       $N00031                    100114e4     net.exp
 0002:0000351e       $N00032                    1001151e     net.exp
 0002:0000355e       $N00033                    1001155e     net.exp
 0002:0000358f       $N00034                    1001158f     net.exp
 0002:000035c2       $N00035                    100115c2     net.exp
 0002:000035f2       $N00036                    100115f2     net.exp
 0002:00003627       $N00037                    10011627     net.exp
 0002:0000364a       $N00038                    1001164a     net.exp
 0002:0000367b       $N00039                    1001167b     net.exp
 0002:000036ae       $N00040                    100116ae     net.exp
 0002:000036de       $N00041                    100116de     net.exp
 0002:00003713       $N00042                    10011713     net.exp
 0002:00003736       $N00043                    10011736     net.exp
 0002:0000376e       $N00044                    1001176e     net.exp
 0002:00003790       $N00045                    10011790     net.exp
 0002:000037b9       $N00046                    100117b9     net.exp
 0002:000037e5       $N00047                    100117e5     net.exp
 0002:00003814       $N00048                    10011814     net.exp
 0002:00003846       $N00049                    10011846     net.exp
 0002:0000387b       $N00050                    1001187b     net.exp
 0002:000038b3       $N00051                    100118b3     net.exp
 0002:000038e1       $N00052                    100118e1     net.exp
 0002:00003912       $N00053                    10011912     net.exp
 0002:0000393d       $N00054                    1001193d     net.exp
 0002:0000396b       $N00055                    1001196b     net.exp
 0002:0000399a       $N00056                    1001199a     net.exp
 0002:000039cc       $N00057                    100119cc     net.exp
 0002:000039f3       $N00058                    100119f3     net.exp
 0002:00003a22       $N00059                    10011a22     net.exp
 0002:00003a54       $N00060                    10011a54     net.exp
 0002:00003a7e       $N00061                    10011a7e     net.exp
 0002:00003aab       $N00062                    10011aab     net.exp
 0002:00003ad4       $N00063                    10011ad4     net.exp
 0002:00003b00       $N00064                    10011b00     net.exp
 0002:00003b36       $N00065                    10011b36     net.exp
 0002:00003b6f       $N00066                    10011b6f     net.exp
 0002:00003b97       $N00067                    10011b97     net.exp
 0002:00003bc7       $N00068                    10011bc7     net.exp
 0002:00003bf0       $N00069                    10011bf0     net.exp
 0002:00003c22       $N00070                    10011c22     net.exp
 0002:00003c5b       $N00071                    10011c5b     net.exp
 0002:00003c97       $N00072                    10011c97     net.exp
 0002:00003cd7       $N00073                    10011cd7     net.exp
 0002:00003d1d       $N00074                    10011d1d     net.exp
 0002:00003d64       $N00075                    10011d64     net.exp
 0002:00003da3       $N00076                    10011da3     net.exp
 0002:00003ddc       $N00077                    10011ddc     net.exp
 0002:00003e1c       $N00078                    10011e1c     net.exp
 0002:00003e53       $N00079                    10011e53     net.exp
 0002:00003e8b       $N00080                    10011e8b     net.exp
 0002:00003ec4       $N00081                    10011ec4     net.exp
 0002:00003efc       $N00082                    10011efc     net.exp
 0002:00003f38       $N00083                    10011f38     net.exp
 0002:00003f74       $N00084                    10011f74     net.exp
 0002:00003fac       $N00085                    10011fac     net.exp
 0002:00003fe6       $N00086                    10011fe6     net.exp
 0002:00004027       $N00087                    10012027     net.exp
 0002:0000406a       $N00088                    1001206a     net.exp
 0002:000040b0       $N00089                    100120b0     net.exp
 0002:000040f9       $N00090                    100120f9     net.exp
 0002:0000412d       $N00091                    1001212d     net.exp
 0002:00004165       $N00092                    10012165     net.exp
 0002:0000419f       $N00093                    1001219f     net.exp
 0002:000041d5       $N00094                    100121d5     net.exp
 0002:0000420d       $N00095                    1001220d     net.exp
 0002:00004246       $N00096                    10012246     net.exp
 0002:0000427e       $N00097                    1001227e     net.exp
 0002:000042b9       $N00098                    100122b9     net.exp
 0002:000042f1       $N00099                    100122f1     net.exp
 0002:00004332       $N00100                    10012332     net.exp
 0002:00004372       $N00101                    10012372     net.exp
 0002:000043ac       $N00102                    100123ac     net.exp
 0002:000043de       $N00103                    100123de     net.exp
 0002:00004411       $N00104                    10012411     net.exp
 0002:0000444b       $N00105                    1001244b     net.exp
 0002:00004486       $N00106                    10012486     net.exp
 0002:000044bf       $N00107                    100124bf     net.exp
 0002:000044e8       $N00108                    100124e8     net.exp
 0002:00004526       $N00109                    10012526     net.exp
 0002:00004559       $N00110                    10012559     net.exp
 0002:00004593       $N00111                    10012593     net.exp
 0002:000045ce       $N00112                    100125ce     net.exp
 0002:00004607       $N00113                    10012607     net.exp
 0002:0000462c       $N00114                    1001262c     net.exp
 0002:00004651       $N00115                    10012651     net.exp
 0002:00004685       $N00116                    10012685     net.exp
 0002:000046c2       $N00117                    100126c2     net.exp
 0002:00004702       $N00118                    10012702     net.exp
 0002:0000473b       $N00119                    1001273b     net.exp
 0002:00004769       $N00120                    10012769     net.exp
 0002:000047b7       $N00121                    100127b7     net.exp
 0002:000047fd       $N00122                    100127fd     net.exp
 0002:00004840       $N00123                    10012840     net.exp
 0002:0000488a       $N00124                    1001288a     net.exp
 0002:000048db       $N00125                    100128db     net.exp
 0002:000048e8       $N00126                    100128e8     net.exp
 0002:000048f6       $N00127                    100128f6     net.exp
 0002:00004913       $N00128                    10012913     net.exp
 0002:0000492e       $N00129                    1001292e     net.exp
 0002:00004941       $N00130                    10012941     net.exp
 0002:0000495f       $N00131                    1001295f     net.exp
 0002:00004977       $N00132                    10012977     net.exp
 0002:00004991       $N00133                    10012991     net.exp
 0002:000049a4       $N00134                    100129a4     net.exp
 0002:000049c6       $N00135                    100129c6     net.exp
 0002:000049e4       $N00136                    100129e4     net.exp
 0002:000049f7       $N00137                    100129f7     net.exp
 0002:00004a08       $N00138                    10012a08     net.exp
 0002:00004a19       $N00139                    10012a19     net.exp
 0002:00004a28       $N00140                    10012a28     net.exp
 0002:00004a38       $N00141                    10012a38     net.exp
 0002:00004a4e       $N00142                    10012a4e     net.exp
 0002:00004dc4       .idata$6                   10012dc4     ws2_32:WS2_32.dll
 0002:00004e1e       .idata$6                   10012e1e     jvm:jvm.dll
 0002:00004f60       .idata$6                   10012f60     java:java.dll
 0002:00004f9c       .idata$6                   10012f9c     advapi32:ADVAPI32.dll
 0002:0000523e       .idata$6                   1001323e     kernel32:KERNEL32.dll
 0002:000052ae       .idata$6                   100132ae     vcruntime:VCRUNTIME140.dll
 0002:00005486       .idata$6                   10013486     ucrt:api-ms-win-crt-string-l1-1-0.dll
 0002:000054a8       .idata$6                   100134a8     ucrt:api-ms-win-crt-stdio-l1-1-0.dll
 0002:000054c8       .idata$6                   100134c8     ucrt:api-ms-win-crt-heap-l1-1-0.dll
 0002:000054e8       .idata$6                   100134e8     ucrt:api-ms-win-crt-runtime-l1-1-0.dll
 0003:00000000       _tcp_level                 10014000     TwoStacksPlainSocketImpl.obj
 0003:0000000c       ?default_tos@?1??NET_GetDefaultTOS@@9@9 1001400c     net_util_md.obj
 0003:00000010       ?opts@?1??NET_MapSocketOption@@9@9 10014010     net_util_md.obj
 0003:000000f8       _proxy_class               100140f8     DefaultProxySelector.obj
 0003:000000fc       _isaddr_class              100140fc     DefaultProxySelector.obj
 0003:00000100       _ptype_class               10014100     DefaultProxySelector.obj
 0003:00000104       _isaddr_createUnresolvedID 10014104     DefaultProxySelector.obj
 0003:00000108       _proxy_ctrID               10014108     DefaultProxySelector.obj
 0003:0000010c       _pr_no_proxyID             1001410c     DefaultProxySelector.obj
 0003:00000110       _ptype_httpID              10014110     DefaultProxySelector.obj
 0003:00000114       _ptype_socksID             10014114     DefaultProxySelector.obj
 0003:00000118       _IO_fd_fdID                10014118     DualStackPlainDatagramSocketImpl.obj
 0003:0000011c       _pdsi_fdID                 1001411c     DualStackPlainDatagramSocketImpl.obj
 0003:00000120       _isa_class                 10014120     DualStackPlainSocketImpl.obj
 0003:00000124       _isa_ctorID                10014124     DualStackPlainSocketImpl.obj
 0003:00000128       _ia4_initialized           10014128     Inet4Address.obj
 0003:0000012c       _ia6_initialized           1001412c     Inet6Address.obj
 0003:00000130       _ia_initialized            10014130     InetAddress.obj
 0003:00000134       _ntlm_ctxHandleID          10014134     NTLMAuthSequence.obj
 0003:00000138       _ntlm_crdHandleID          10014138     NTLMAuthSequence.obj
 0003:0000013c       _status_seqCompleteID      1001413c     NTLMAuthSequence.obj
 0003:00000140       _fn_CoInternetCreateSecurityManager 10014140     NTLMAuthentication.obj
 0003:00000144       _searchlistID              10014144     ResolverConfigurationImpl.obj
 0003:00000148       _nameserversID             10014148     ResolverConfigurationImpl.obj
 0003:0000014c       _IO_fd_fdID                1001414c     SocketInputStream.obj
 0003:00000150       _IO_fd_fdID                10014150     SocketOutputStream.obj
 0003:00000154       _IO_fd_fdID                10014154     TwoStacksPlainDatagramSocketImpl.obj
 0003:00000158       _pdsi_trafficClassID       10014158     TwoStacksPlainDatagramSocketImpl.obj
 0003:0000015c       _ia4_clazz                 1001415c     TwoStacksPlainDatagramSocketImpl.obj
 0003:00000160       _ia4_ctor                  10014160     TwoStacksPlainDatagramSocketImpl.obj
 0003:00000164       _sizeCheckLock             10014164     TwoStacksPlainDatagramSocketImpl.obj
 0003:0000017c       _xp_or_later               1001417c     TwoStacksPlainDatagramSocketImpl.obj
 0003:00000180       _w2k_or_later              10014180     TwoStacksPlainDatagramSocketImpl.obj
 0003:00000184       ?i_class@?1??createInteger@@9@9 10014184     TwoStacksPlainDatagramSocketImpl.obj
 0003:00000188       ?i_ctrID@?1??createInteger@@9@9 10014188     TwoStacksPlainDatagramSocketImpl.obj
 0003:0000018c       ?b_class@?1??createBoolean@@9@9 1001418c     TwoStacksPlainDatagramSocketImpl.obj
 0003:00000190       ?b_ctrID@?1??createBoolean@@9@9 10014190     TwoStacksPlainDatagramSocketImpl.obj
 0003:00000194       ?initDone@?1??exceedSizeLimit@@9@9 10014194     TwoStacksPlainDatagramSocketImpl.obj
 0003:00000195       ?is95or98@?1??exceedSizeLimit@@9@9 10014195     TwoStacksPlainDatagramSocketImpl.obj
 0003:00000196       ?initDone@?1??supportPortUnreachable@@9@9 10014196     TwoStacksPlainDatagramSocketImpl.obj
 0003:00000197       ?portUnreachableSupported@?1??supportPortUnreachable@@9@9 10014197     TwoStacksPlainDatagramSocketImpl.obj
 0003:00000198       ?maxmsg@?1??exceedSizeLimit@@9@9 10014198     TwoStacksPlainDatagramSocketImpl.obj
 0003:0000019c       ?addrList@?1??exceedSizeLimit@@9@9 1001419c     TwoStacksPlainDatagramSocketImpl.obj
 0003:000001a0       ?ni_addrsID@?1??getInetAddrFromIf@@9@9 100141a0     TwoStacksPlainDatagramSocketImpl.obj
 0003:000001a4       ?ni_indexID@?1??getIndexFromIf@@9@9 100141a4     TwoStacksPlainDatagramSocketImpl.obj
 0003:000001a8       ?ni_class@?3??setMulticastInterface@@9@9 100141a8     TwoStacksPlainDatagramSocketImpl.obj
 0003:000001ac       ?ni_indexID@?BB@??setMulticastInterface@@9@9 100141ac     TwoStacksPlainDatagramSocketImpl.obj
 0003:000001b0       ?inet4_class@?1??getIPv4NetworkInterface@@9@9 100141b0     TwoStacksPlainDatagramSocketImpl.obj
 0003:000001b4       ?inet4_ctrID@?1??getIPv4NetworkInterface@@9@9 100141b4     TwoStacksPlainDatagramSocketImpl.obj
 0003:000001b8       ?ni_class@?1??getIPv4NetworkInterface@@9@9 100141b8     TwoStacksPlainDatagramSocketImpl.obj
 0003:000001bc       ?ni_ctrID@?1??getIPv4NetworkInterface@@9@9 100141bc     TwoStacksPlainDatagramSocketImpl.obj
 0003:000001c0       ?ni_indexID@?1??getIPv4NetworkInterface@@9@9 100141c0     TwoStacksPlainDatagramSocketImpl.obj
 0003:000001c4       ?ni_addrsID@?1??getIPv4NetworkInterface@@9@9 100141c4     TwoStacksPlainDatagramSocketImpl.obj
 0003:000001c8       ?ni_class@?3??getMulticastInterface@@9@9 100141c8     TwoStacksPlainDatagramSocketImpl.obj
 0003:000001cc       ?ni_ctrID@?3??getMulticastInterface@@9@9 100141cc     TwoStacksPlainDatagramSocketImpl.obj
 0003:000001d0       ?ni_indexID@?3??getMulticastInterface@@9@9 100141d0     TwoStacksPlainDatagramSocketImpl.obj
 0003:000001d4       ?ni_addrsID@?3??getMulticastInterface@@9@9 100141d4     TwoStacksPlainDatagramSocketImpl.obj
 0003:000001d8       ?ia_class@?3??getMulticastInterface@@9@9 100141d8     TwoStacksPlainDatagramSocketImpl.obj
 0003:000001dc       ?ia_anyLocalAddressID@?3??getMulticastInterface@@9@9 100141dc     TwoStacksPlainDatagramSocketImpl.obj
 0003:000001e0       _IO_fd_fdID                100141e0     TwoStacksPlainSocketImpl.obj
 0003:000001e4       ?inet4Cls@?1??Java_java_net_TwoStacksPlainSocketImpl_socketAccept@@9@9 100141e4     TwoStacksPlainSocketImpl.obj
 0003:000001e8       ?inet6Cls@?1??Java_java_net_TwoStacksPlainSocketImpl_socketAccept@@9@9 100141e8     TwoStacksPlainSocketImpl.obj
 0003:000001ec       _IPv6_available            100141ec     net_util.obj
 0003:000001f0       _initialized               100141f0     net_util.obj
 0003:000001f4       ?cls@?1??NET_ThrowSocketException@@9@9 100141f4     net_util_md.obj
 0003:0000021c       ?__proc_attached@@3HA      1001421c     MSVCRT:dll_dllmain.obj
 0003:00000220       _GS_ExceptionRecord        10014220     MSVCRT:gs_report.obj
 0003:00000270       _GS_ContextRecord          10014270     MSVCRT:gs_report.obj
 0003:00000550       ?is_initialized_as_dll@@3_NA 10014550     MSVCRT:utility.obj
 0003:00000551       ?module_local_atexit_table_initialized@@3_NA 10014551     MSVCRT:utility.obj
 0003:00000554       ?module_local_atexit_table@@3U_onexit_table_t@@A 10014554     MSVCRT:utility.obj
 0003:00000560       ?module_local_at_quick_exit_table@@3U_onexit_table_t@@A 10014560     MSVCRT:utility.obj
 0004:00000060       $R000000                   10015060     net.dll.res
